** EXPERIMENTAL (HLL) ** Open Watcom Linker Version 1.6beta1 Limited Availability
Portions Copyright (c) 1985-2002 Sybase, Inc. All Rights Reserved.
Created on:       10/10/20 19:59:58
Executable Image: httpd.dll
creating an OS/2 EMX dynamic link library


                        +------------+
                        |   Groups   |
                        +------------+

Group                           Address              Size
=====                           =======              ====

CGROUP                          0001:00000000        0007a740
DGROUP                          0002:00000000        00003ea0



                        +--------------+
                        |   Segments   |
                        +--------------+

Segment                Class          Group          Address         Size
=======                =====          =====          =======         ====

TEXT32                 CODE           CGROUP         0001:00000000   0007a740
________TEXT           CODE           CGROUP         0001:0007a740   00000000
DATA32                 DATA           DGROUP         0002:00000000   00002b60
SET1__os2dll           DATA           DGROUP         0002:00002b60   00000004
SET2__os2dll           DATA           DGROUP         0002:00002b64   00000000
SET3__os2dll           DATA           DGROUP         0002:00002b64   00000004
SET1___CTOR_LIST__     DATA           DGROUP         0002:00002b68   00000004
SET2___CTOR_LIST__     DATA           DGROUP         0002:00002b6c   00000000
SET3___CTOR_LIST__     DATA           DGROUP         0002:00002b6c   00000004
SET1___DTOR_LIST__     DATA           DGROUP         0002:00002b70   00000004
SET2___DTOR_LIST__     DATA           DGROUP         0002:00002b74   00000000
SET3___DTOR_LIST__     DATA           DGROUP         0002:00002b74   00000004
SET1___crtinit1__      DATA           DGROUP         0002:00002b78   00000004
SET2___crtinit1__      DATA           DGROUP         0002:00002b7c   00000000
SET3___crtinit1__      DATA           DGROUP         0002:00002b7c   00000004
SET1___crtexit1__      DATA           DGROUP         0002:00002b80   00000004
SET2___crtexit1__      DATA           DGROUP         0002:00002b84   00000000
SET3___crtexit1__      DATA           DGROUP         0002:00002b84   00000004
SET1___eh_frame__      DATA           DGROUP         0002:00002b88   00000004
SET2___eh_frame__      DATA           DGROUP         0002:00002b8c   00000014
SET3___eh_frame__      DATA           DGROUP         0002:00002ba0   00000004
SET1___eh_init__       DATA           DGROUP         0002:00002ba4   00000004
SET2___eh_init__       DATA           DGROUP         0002:00002ba8   00000004
SET3___eh_init__       DATA           DGROUP         0002:00002bac   00000004
SET1___eh_term__       DATA           DGROUP         0002:00002bb0   00000004
SET2___eh_term__       DATA           DGROUP         0002:00002bb4   00000004
SET3___eh_term__       DATA           DGROUP         0002:00002bb8   00000004
SET1___fork_parent1__  DATA           DGROUP         0002:00002bbc   00000004
SET2___fork_parent1__  DATA           DGROUP         0002:00002bc0   00000000
SET3___fork_parent1__  DATA           DGROUP         0002:00002bc0   00000004
SET1___fork_child1__   DATA           DGROUP         0002:00002bc4   00000004
SET2___fork_child1__   DATA           DGROUP         0002:00002bc8   00000000
SET3___fork_child1__   DATA           DGROUP         0002:00002bc8   00000004
________DATA           DATA           DGROUP         0002:00002bd0   00000000
BSS32                  BSS            DGROUP         0002:00002bd0   000011f0
c_common               BSS            DGROUP         0002:00003dc0   000000e0
________BSS            BSS            DGROUP         0002:00003ea0   00000000


                        +----------------+
                        |   Memory Map   |
                        +----------------+

* = unreferenced symbol
+ = symbol only referenced locally

Address        Symbol
=======        ======

Module: U:\usr\lib\dll0.obj({standard input})
0001:00000000* __text
0002:00000000* __data
0002:00000000* ___data_start
0002:00002bd0* ___bss_start
0002:00002b60+ __os2dll
0002:00002b68  ___CTOR_LIST__
0002:00002b70  ___DTOR_LIST__
0002:00002b78* ___crtinit1__
0002:00002b80* ___crtexit1__
0002:00002b88  ___eh_frame__
0002:00002ba4  ___eh_init__
0002:00002bb0  ___eh_term__
0002:00002bbc+ ___fork_parent1__
0002:00002bc4+ ___fork_child1__
Module: U:\dev\httpd-2.2.17\buildmark.o(buildmark.o)
0001:000000a0  _ap_get_server_built
Module: U:\dev\httpd-2.2.17\server\exports.o(exports.o)
0002:00000050* _ap_hack_apr_allocator_create
0002:00000054* _ap_hack_apr_allocator_destroy
0002:00000058* _ap_hack_apr_allocator_alloc
0002:0000005c* _ap_hack_apr_allocator_free
0002:00000060* _ap_hack_apr_allocator_owner_set
0002:00000064* _ap_hack_apr_allocator_owner_get
0002:00000068* _ap_hack_apr_allocator_max_free_set
0002:0000006c* _ap_hack_apr_allocator_mutex_set
0002:00000070* _ap_hack_apr_allocator_mutex_get
0002:00000074* _ap_hack_apr_atomic_init
0002:00000078* _ap_hack_apr_atomic_read32
0002:0000007c* _ap_hack_apr_atomic_set32
0002:00000080* _ap_hack_apr_atomic_add32
0002:00000084* _ap_hack_apr_atomic_sub32
0002:00000088* _ap_hack_apr_atomic_inc32
0002:0000008c* _ap_hack_apr_atomic_dec32
0002:00000090* _ap_hack_apr_atomic_cas32
0002:00000094* _ap_hack_apr_atomic_xchg32
0002:00000098* _ap_hack_apr_atomic_casptr
0002:0000009c* _ap_hack_apr_atomic_xchgptr
0002:000000a0* _ap_hack_apr_base64_encode_len
0002:000000a4* _ap_hack_apr_base64_encode
0002:000000a8* _ap_hack_apr_base64_encode_binary
0002:000000ac* _ap_hack_apr_base64_decode_len
0002:000000b0* _ap_hack_apr_base64_decode
0002:000000b4* _ap_hack_apr_base64_decode_binary
0002:000000b8* _ap_hack_apr_brigade_create
0002:000000bc* _ap_hack_apr_brigade_destroy
0002:000000c0* _ap_hack_apr_brigade_cleanup
0002:000000c4* _ap_hack_apr_brigade_split_ex
0002:000000c8* _ap_hack_apr_brigade_split
0002:000000cc* _ap_hack_apr_brigade_partition
0002:000000d0* _ap_hack_apr_brigade_length
0002:000000d4* _ap_hack_apr_brigade_flatten
0002:000000d8* _ap_hack_apr_brigade_pflatten
0002:000000dc* _ap_hack_apr_brigade_split_line
0002:000000e0* _ap_hack_apr_brigade_to_iovec
0002:000000e4* _ap_hack_apr_brigade_vputstrs
0002:000000e8* _ap_hack_apr_brigade_write
0002:000000ec* _ap_hack_apr_brigade_writev
0002:000000f0* _ap_hack_apr_brigade_puts
0002:000000f4* _ap_hack_apr_brigade_putc
0002:000000f8* _ap_hack_apr_brigade_putstrs
0002:000000fc* _ap_hack_apr_brigade_printf
0002:00000100* _ap_hack_apr_brigade_vprintf
0002:00000104* _ap_hack_apr_brigade_insert_file
0002:00000108* _ap_hack_apr_bucket_alloc_create
0002:0000010c* _ap_hack_apr_bucket_alloc_create_ex
0002:00000110* _ap_hack_apr_bucket_alloc_destroy
0002:00000114* _ap_hack_apr_bucket_alloc
0002:00000118* _ap_hack_apr_bucket_free
0002:0000011c* _ap_hack_apr_bucket_setaside_noop
0002:00000120* _ap_hack_apr_bucket_setaside_notimpl
0002:00000124* _ap_hack_apr_bucket_split_notimpl
0002:00000128* _ap_hack_apr_bucket_copy_notimpl
0002:0000012c* _ap_hack_apr_bucket_destroy_noop
0002:00000130* _ap_hack_apr_bucket_simple_split
0002:00000134* _ap_hack_apr_bucket_simple_copy
0002:00000138* _ap_hack_apr_bucket_shared_make
0002:0000013c* _ap_hack_apr_bucket_shared_destroy
0002:00000140* _ap_hack_apr_bucket_shared_split
0002:00000144* _ap_hack_apr_bucket_shared_copy
0002:00000148* _ap_hack_apr_bucket_eos_create
0002:0000014c* _ap_hack_apr_bucket_eos_make
0002:00000150* _ap_hack_apr_bucket_flush_create
0002:00000154* _ap_hack_apr_bucket_flush_make
0002:00000158* _ap_hack_apr_bucket_immortal_create
0002:0000015c* _ap_hack_apr_bucket_immortal_make
0002:00000160* _ap_hack_apr_bucket_transient_create
0002:00000164* _ap_hack_apr_bucket_transient_make
0002:00000168* _ap_hack_apr_bucket_heap_create
0002:0000016c* _ap_hack_apr_bucket_heap_make
0002:00000170* _ap_hack_apr_bucket_pool_create
0002:00000174* _ap_hack_apr_bucket_pool_make
0002:00000178* _ap_hack_apr_bucket_socket_create
0002:0000017c* _ap_hack_apr_bucket_socket_make
0002:00000180* _ap_hack_apr_bucket_pipe_create
0002:00000184* _ap_hack_apr_bucket_pipe_make
0002:00000188* _ap_hack_apr_bucket_file_create
0002:0000018c* _ap_hack_apr_bucket_file_make
0002:00000190* _ap_hack_apr_bucket_file_enable_mmap
0002:00000194* _ap_hack_apr_date_checkmask
0002:00000198* _ap_hack_apr_date_parse_http
0002:0000019c* _ap_hack_apr_date_parse_rfc
0002:000001a0* _ap_hack_apr_dbd_init
0002:000001a4* _ap_hack_apr_dbd_get_driver
0002:000001a8* _ap_hack_apr_dbd_open_ex
0002:000001ac* _ap_hack_apr_dbd_open
0002:000001b0* _ap_hack_apr_dbd_close
0002:000001b4* _ap_hack_apr_dbd_name
0002:000001b8* _ap_hack_apr_dbd_native_handle
0002:000001bc* _ap_hack_apr_dbd_check_conn
0002:000001c0* _ap_hack_apr_dbd_set_dbname
0002:000001c4* _ap_hack_apr_dbd_transaction_start
0002:000001c8* _ap_hack_apr_dbd_transaction_end
0002:000001cc* _ap_hack_apr_dbd_transaction_mode_get
0002:000001d0* _ap_hack_apr_dbd_transaction_mode_set
0002:000001d4* _ap_hack_apr_dbd_query
0002:000001d8* _ap_hack_apr_dbd_select
0002:000001dc* _ap_hack_apr_dbd_num_cols
0002:000001e0* _ap_hack_apr_dbd_num_tuples
0002:000001e4* _ap_hack_apr_dbd_get_row
0002:000001e8* _ap_hack_apr_dbd_get_entry
0002:000001ec* _ap_hack_apr_dbd_get_name
0002:000001f0* _ap_hack_apr_dbd_error
0002:000001f4* _ap_hack_apr_dbd_escape
0002:000001f8* _ap_hack_apr_dbd_prepare
0002:000001fc* _ap_hack_apr_dbd_pquery
0002:00000200* _ap_hack_apr_dbd_pselect
0002:00000204* _ap_hack_apr_dbd_pvquery
0002:00000208* _ap_hack_apr_dbd_pvselect
0002:0000020c* _ap_hack_apr_dbd_pbquery
0002:00000210* _ap_hack_apr_dbd_pbselect
0002:00000214* _ap_hack_apr_dbd_pvbquery
0002:00000218* _ap_hack_apr_dbd_pvbselect
0002:0000021c* _ap_hack_apr_dbd_datum_get
0002:00000220* _ap_hack_apr_dbm_open_ex
0002:00000224* _ap_hack_apr_dbm_open
0002:00000228* _ap_hack_apr_dbm_close
0002:0000022c* _ap_hack_apr_dbm_fetch
0002:00000230* _ap_hack_apr_dbm_store
0002:00000234* _ap_hack_apr_dbm_delete
0002:00000238* _ap_hack_apr_dbm_exists
0002:0000023c* _ap_hack_apr_dbm_firstkey
0002:00000240* _ap_hack_apr_dbm_nextkey
0002:00000244* _ap_hack_apr_dbm_freedatum
0002:00000248* _ap_hack_apr_dbm_geterror
0002:0000024c* _ap_hack_apr_dbm_get_usednames_ex
0002:00000250* _ap_hack_apr_dbm_get_usednames
0002:00000254* _ap_hack_apr_dso_load
0002:00000258* _ap_hack_apr_dso_unload
0002:0000025c* _ap_hack_apr_dso_sym
0002:00000260* _ap_hack_apr_dso_error
0002:00000264* _ap_hack_apr_env_get
0002:00000268* _ap_hack_apr_env_set
0002:0000026c* _ap_hack_apr_env_delete
0002:00000270* _ap_hack_apr_strerror
0002:00000274* _ap_hack_apr_stat
0002:00000278* _ap_hack_apr_dir_open
0002:0000027c* _ap_hack_apr_dir_close
0002:00000280* _ap_hack_apr_dir_read
0002:00000284* _ap_hack_apr_dir_rewind
0002:00000288* _ap_hack_apr_filepath_root
0002:0000028c* _ap_hack_apr_filepath_merge
0002:00000290* _ap_hack_apr_filepath_list_split
0002:00000294* _ap_hack_apr_filepath_list_merge
0002:00000298* _ap_hack_apr_filepath_get
0002:0000029c* _ap_hack_apr_filepath_set
0002:000002a0* _ap_hack_apr_filepath_encoding
0002:000002a4* _ap_hack_apr_file_open
0002:000002a8* _ap_hack_apr_file_close
0002:000002ac* _ap_hack_apr_file_remove
0002:000002b0* _ap_hack_apr_file_rename
0002:000002b4* _ap_hack_apr_file_link
0002:000002b8* _ap_hack_apr_file_copy
0002:000002bc* _ap_hack_apr_file_append
0002:000002c0* _ap_hack_apr_file_eof
0002:000002c4* _ap_hack_apr_file_open_stderr
0002:000002c8* _ap_hack_apr_file_open_stdout
0002:000002cc* _ap_hack_apr_file_open_stdin
0002:000002d0* _ap_hack_apr_file_open_flags_stderr
0002:000002d4* _ap_hack_apr_file_open_flags_stdout
0002:000002d8* _ap_hack_apr_file_open_flags_stdin
0002:000002dc* _ap_hack_apr_file_read
0002:000002e0* _ap_hack_apr_file_write
0002:000002e4* _ap_hack_apr_file_writev
0002:000002e8* _ap_hack_apr_file_read_full
0002:000002ec* _ap_hack_apr_file_write_full
0002:000002f0* _ap_hack_apr_file_writev_full
0002:000002f4* _ap_hack_apr_file_putc
0002:000002f8* _ap_hack_apr_file_getc
0002:000002fc* _ap_hack_apr_file_ungetc
0002:00000300* _ap_hack_apr_file_gets
0002:00000304* _ap_hack_apr_file_puts
0002:00000308* _ap_hack_apr_file_flush
0002:0000030c* _ap_hack_apr_file_sync
0002:00000310* _ap_hack_apr_file_datasync
0002:00000314* _ap_hack_apr_file_dup
0002:00000318* _ap_hack_apr_file_dup2
0002:0000031c* _ap_hack_apr_file_setaside
0002:00000320* _ap_hack_apr_file_buffer_set
0002:00000324* _ap_hack_apr_file_buffer_size_get
0002:00000328* _ap_hack_apr_file_seek
0002:0000032c* _ap_hack_apr_file_pipe_create
0002:00000330* _ap_hack_apr_file_pipe_create_ex
0002:00000334* _ap_hack_apr_file_namedpipe_create
0002:00000338* _ap_hack_apr_file_pipe_timeout_get
0002:0000033c* _ap_hack_apr_file_pipe_timeout_set
0002:00000340* _ap_hack_apr_file_lock
0002:00000344* _ap_hack_apr_file_unlock
0002:00000348* _ap_hack_apr_file_name_get
0002:0000034c* _ap_hack_apr_file_data_get
0002:00000350* _ap_hack_apr_file_data_set
0002:00000354* _ap_hack_apr_file_printf
0002:00000358* _ap_hack_apr_file_perms_set
0002:0000035c* _ap_hack_apr_file_attrs_set
0002:00000360* _ap_hack_apr_file_mtime_set
0002:00000364* _ap_hack_apr_dir_make
0002:00000368* _ap_hack_apr_dir_make_recursive
0002:0000036c* _ap_hack_apr_dir_remove
0002:00000370* _ap_hack_apr_file_info_get
0002:00000374* _ap_hack_apr_file_trunc
0002:00000378* _ap_hack_apr_file_flags_get
0002:0000037c* _ap_hack_apr_file_pool_get
0002:00000380* _ap_hack_apr_file_inherit_set
0002:00000384* _ap_hack_apr_file_inherit_unset
0002:00000388* _ap_hack_apr_file_mktemp
0002:0000038c* _ap_hack_apr_temp_dir_get
0002:00000390* _ap_hack_apr_fnmatch
0002:00000394* _ap_hack_apr_fnmatch_test
0002:00000398* _ap_hack_apr_match_glob
0002:0000039c* _ap_hack_apr_initialize
0002:000003a0* _ap_hack_apr_app_initialize
0002:000003a4* _ap_hack_apr_terminate
0002:000003a8* _ap_hack_apr_terminate2
0002:000003ac* _ap_hack_apr_generate_random_bytes
0002:000003b0* _ap_hack_apr_getopt_init
0002:000003b4* _ap_hack_apr_getopt
0002:000003b8* _ap_hack_apr_getopt_long
0002:000003bc* _ap_hack_apr_hashfunc_default
0002:000003c0* _ap_hack_apr_hash_make
0002:000003c4* _ap_hack_apr_hash_make_custom
0002:000003c8* _ap_hack_apr_hash_copy
0002:000003cc* _ap_hack_apr_hash_set
0002:000003d0* _ap_hack_apr_hash_get
0002:000003d4* _ap_hack_apr_hash_first
0002:000003d8* _ap_hack_apr_hash_next
0002:000003dc* _ap_hack_apr_hash_this
0002:000003e0* _ap_hack_apr_hash_count
0002:000003e4* _ap_hack_apr_hash_clear
0002:000003e8* _ap_hack_apr_hash_overlay
0002:000003ec* _ap_hack_apr_hash_merge
0002:000003f0* _ap_hack_apr_hash_do
0002:000003f4* _ap_hack_apr_hash_pool_get
0002:000003f8* _ap_hack_apr_hook_sort_register
0002:000003fc* _ap_hack_apr_hook_sort_all
0002:00000400* _ap_hack_apr_hook_debug_show
0002:00000404* _ap_hack_apr_hook_deregister_all
0002:00000408* _ap_hack_apr_filepath_name_get
0002:0000040c* _ap_hack_apr_vformatter
0002:00000410* _ap_hack_apr_password_get
0002:00000414* _ap_hack_apr_md4_init
0002:00000418* _ap_hack_apr_md4_set_xlate
0002:0000041c* _ap_hack_apr_md4_update
0002:00000420* _ap_hack_apr_md4_final
0002:00000424* _ap_hack_apr_md4
0002:00000428* _ap_hack_apr_md5_init
0002:0000042c* _ap_hack_apr_md5_set_xlate
0002:00000430* _ap_hack_apr_md5_update
0002:00000434* _ap_hack_apr_md5_final
0002:00000438* _ap_hack_apr_md5
0002:0000043c* _ap_hack_apr_md5_encode
0002:00000440* _ap_hack_apr_password_validate
0002:00000444* _ap_hack_apr_memcache_hash
0002:00000448* _ap_hack_apr_memcache_hash_crc32
0002:0000044c* _ap_hack_apr_memcache_hash_default
0002:00000450* _ap_hack_apr_memcache_find_server_hash
0002:00000454* _ap_hack_apr_memcache_find_server_hash_default
0002:00000458* _ap_hack_apr_memcache_add_server
0002:0000045c* _ap_hack_apr_memcache_find_server
0002:00000460* _ap_hack_apr_memcache_enable_server
0002:00000464* _ap_hack_apr_memcache_disable_server
0002:00000468* _ap_hack_apr_memcache_server_create
0002:0000046c* _ap_hack_apr_memcache_create
0002:00000470* _ap_hack_apr_memcache_getp
0002:00000474* _ap_hack_apr_memcache_add_multget_key
0002:00000478* _ap_hack_apr_memcache_multgetp
0002:0000047c* _ap_hack_apr_memcache_set
0002:00000480* _ap_hack_apr_memcache_add
0002:00000484* _ap_hack_apr_memcache_replace
0002:00000488* _ap_hack_apr_memcache_delete
0002:0000048c* _ap_hack_apr_memcache_incr
0002:00000490* _ap_hack_apr_memcache_decr
0002:00000494* _ap_hack_apr_memcache_version
0002:00000498* _ap_hack_apr_memcache_stats
0002:0000049c* _ap_hack_apr_socket_create
0002:000004a0* _ap_hack_apr_socket_shutdown
0002:000004a4* _ap_hack_apr_socket_close
0002:000004a8* _ap_hack_apr_socket_bind
0002:000004ac* _ap_hack_apr_socket_listen
0002:000004b0* _ap_hack_apr_socket_accept
0002:000004b4* _ap_hack_apr_socket_connect
0002:000004b8* _ap_hack_apr_socket_atreadeof
0002:000004bc* _ap_hack_apr_sockaddr_info_get
0002:000004c0* _ap_hack_apr_getnameinfo
0002:000004c4* _ap_hack_apr_parse_addr_port
0002:000004c8* _ap_hack_apr_gethostname
0002:000004cc* _ap_hack_apr_socket_data_get
0002:000004d0* _ap_hack_apr_socket_data_set
0002:000004d4* _ap_hack_apr_socket_send
0002:000004d8* _ap_hack_apr_socket_sendv
0002:000004dc* _ap_hack_apr_socket_sendto
0002:000004e0* _ap_hack_apr_socket_recvfrom
0002:000004e4* _ap_hack_apr_socket_recv
0002:000004e8* _ap_hack_apr_socket_opt_set
0002:000004ec* _ap_hack_apr_socket_timeout_set
0002:000004f0* _ap_hack_apr_socket_opt_get
0002:000004f4* _ap_hack_apr_socket_timeout_get
0002:000004f8* _ap_hack_apr_socket_atmark
0002:000004fc* _ap_hack_apr_socket_addr_get
0002:00000500* _ap_hack_apr_sockaddr_ip_get
0002:00000504* _ap_hack_apr_sockaddr_ip_getbuf
0002:00000508* _ap_hack_apr_sockaddr_equal
0002:0000050c* _ap_hack_apr_socket_type_get
0002:00000510* _ap_hack_apr_getservbyname
0002:00000514* _ap_hack_apr_ipsubnet_create
0002:00000518* _ap_hack_apr_ipsubnet_test
0002:0000051c* _ap_hack_apr_socket_protocol_get
0002:00000520* _ap_hack_apr_socket_pool_get
0002:00000524* _ap_hack_apr_socket_inherit_set
0002:00000528* _ap_hack_apr_socket_inherit_unset
0002:0000052c* _ap_hack_apr_optional_hook_add
0002:00000530* _ap_hack_apr_optional_hook_get
0002:00000534* _ap_hack_apr_dynamic_fn_register
0002:00000538* _ap_hack_apr_dynamic_fn_retrieve
0002:0000053c* _ap_hack_apr_pollset_create
0002:00000540* _ap_hack_apr_pollset_create_ex
0002:00000544* _ap_hack_apr_pollset_destroy
0002:00000548* _ap_hack_apr_pollset_add
0002:0000054c* _ap_hack_apr_pollset_remove
0002:00000550* _ap_hack_apr_pollset_poll
0002:00000554* _ap_hack_apr_poll
0002:00000558* _ap_hack_apr_pollcb_create
0002:0000055c* _ap_hack_apr_pollcb_add
0002:00000560* _ap_hack_apr_pollcb_remove
0002:00000564* _ap_hack_apr_pollcb_poll
0002:00000568* _ap_hack_apr_pool_initialize
0002:0000056c* _ap_hack_apr_pool_terminate
0002:00000570* _ap_hack_apr_pool_create_ex
0002:00000574* _ap_hack_apr_pool_create_core_ex
0002:00000578* _ap_hack_apr_pool_create_unmanaged_ex
0002:0000057c* _ap_hack_apr_pool_create_ex_debug
0002:00000580* _ap_hack_apr_pool_create_core_ex_debug
0002:00000584* _ap_hack_apr_pool_create_unmanaged_ex_debug
0002:00000588* _ap_hack_apr_pool_allocator_get
0002:0000058c* _ap_hack_apr_pool_clear
0002:00000590* _ap_hack_apr_pool_clear_debug
0002:00000594* _ap_hack_apr_pool_destroy
0002:00000598* _ap_hack_apr_pool_destroy_debug
0002:0000059c* _ap_hack_apr_palloc
0002:000005a0* _ap_hack_apr_palloc_debug
0002:000005a4* _ap_hack_apr_pcalloc_debug
0002:000005a8* _ap_hack_apr_pool_abort_set
0002:000005ac* _ap_hack_apr_pool_abort_get
0002:000005b0* _ap_hack_apr_pool_parent_get
0002:000005b4* _ap_hack_apr_pool_is_ancestor
0002:000005b8* _ap_hack_apr_pool_tag
0002:000005bc* _ap_hack_apr_pool_userdata_set
0002:000005c0* _ap_hack_apr_pool_userdata_setn
0002:000005c4* _ap_hack_apr_pool_userdata_get
0002:000005c8* _ap_hack_apr_pool_cleanup_register
0002:000005cc* _ap_hack_apr_pool_pre_cleanup_register
0002:000005d0* _ap_hack_apr_pool_cleanup_kill
0002:000005d4* _ap_hack_apr_pool_child_cleanup_set
0002:000005d8* _ap_hack_apr_pool_cleanup_run
0002:000005dc* _ap_hack_apr_pool_cleanup_null
0002:000005e0* _ap_hack_apr_pool_cleanup_for_exec
0002:000005e4* _ap_hack_apr_os_file_get
0002:000005e8* _ap_hack_apr_os_dir_get
0002:000005ec* _ap_hack_apr_os_sock_get
0002:000005f0* _ap_hack_apr_os_proc_mutex_get
0002:000005f4* _ap_hack_apr_os_exp_time_get
0002:000005f8* _ap_hack_apr_os_imp_time_get
0002:000005fc* _ap_hack_apr_os_shm_get
0002:00000600* _ap_hack_apr_os_thread_get
0002:00000604* _ap_hack_apr_os_threadkey_get
0002:00000608* _ap_hack_apr_os_thread_put
0002:0000060c* _ap_hack_apr_os_threadkey_put
0002:00000610* _ap_hack_apr_os_thread_current
0002:00000614* _ap_hack_apr_os_thread_equal
0002:00000618* _ap_hack_apr_os_file_put
0002:0000061c* _ap_hack_apr_os_pipe_put
0002:00000620* _ap_hack_apr_os_pipe_put_ex
0002:00000624* _ap_hack_apr_os_dir_put
0002:00000628* _ap_hack_apr_os_sock_put
0002:0000062c* _ap_hack_apr_os_sock_make
0002:00000630* _ap_hack_apr_os_proc_mutex_put
0002:00000634* _ap_hack_apr_os_imp_time_put
0002:00000638* _ap_hack_apr_os_exp_time_put
0002:0000063c* _ap_hack_apr_os_shm_put
0002:00000640* _ap_hack_apr_os_dso_handle_put
0002:00000644* _ap_hack_apr_os_dso_handle_get
0002:00000648* _ap_hack_apr_os_default_encoding
0002:0000064c* _ap_hack_apr_os_locale_encoding
0002:00000650* _ap_hack_apr_proc_mutex_create
0002:00000654* _ap_hack_apr_proc_mutex_child_init
0002:00000658* _ap_hack_apr_proc_mutex_lock
0002:0000065c* _ap_hack_apr_proc_mutex_trylock
0002:00000660* _ap_hack_apr_proc_mutex_unlock
0002:00000664* _ap_hack_apr_proc_mutex_destroy
0002:00000668* _ap_hack_apr_proc_mutex_cleanup
0002:0000066c* _ap_hack_apr_proc_mutex_lockfile
0002:00000670* _ap_hack_apr_proc_mutex_name
0002:00000674* _ap_hack_apr_proc_mutex_defname
0002:00000678* _ap_hack_apr_proc_mutex_pool_get
0002:0000067c* _ap_hack_apr_queue_create
0002:00000680* _ap_hack_apr_queue_push
0002:00000684* _ap_hack_apr_queue_pop
0002:00000688* _ap_hack_apr_queue_trypush
0002:0000068c* _ap_hack_apr_queue_trypop
0002:00000690* _ap_hack_apr_queue_size
0002:00000694* _ap_hack_apr_queue_interrupt_all
0002:00000698* _ap_hack_apr_queue_term
0002:0000069c* _ap_hack_apr_crypto_sha256_new
0002:000006a0* _ap_hack_apr_random_init
0002:000006a4* _ap_hack_apr_random_standard_new
0002:000006a8* _ap_hack_apr_random_add_entropy
0002:000006ac* _ap_hack_apr_random_insecure_bytes
0002:000006b0* _ap_hack_apr_random_secure_bytes
0002:000006b4* _ap_hack_apr_random_barrier
0002:000006b8* _ap_hack_apr_random_secure_ready
0002:000006bc* _ap_hack_apr_random_insecure_ready
0002:000006c0* _ap_hack_apr_random_after_fork
0002:000006c4* _ap_hack_apr_reslist_create
0002:000006c8* _ap_hack_apr_reslist_destroy
0002:000006cc* _ap_hack_apr_reslist_acquire
0002:000006d0* _ap_hack_apr_reslist_release
0002:000006d4* _ap_hack_apr_reslist_timeout_set
0002:000006d8* _ap_hack_apr_reslist_acquired_count
0002:000006dc* _ap_hack_apr_reslist_invalidate
0002:000006e0* _ap_hack_apr_rmm_init
0002:000006e4* _ap_hack_apr_rmm_destroy
0002:000006e8* _ap_hack_apr_rmm_attach
0002:000006ec* _ap_hack_apr_rmm_detach
0002:000006f0* _ap_hack_apr_rmm_malloc
0002:000006f4* _ap_hack_apr_rmm_realloc
0002:000006f8* _ap_hack_apr_rmm_calloc
0002:000006fc* _ap_hack_apr_rmm_free
0002:00000700* _ap_hack_apr_rmm_addr_get
0002:00000704* _ap_hack_apr_rmm_offset_get
0002:00000708* _ap_hack_apr_rmm_overhead_get
0002:0000070c* _ap_hack_apr_sdbm_open
0002:00000710* _ap_hack_apr_sdbm_close
0002:00000714* _ap_hack_apr_sdbm_lock
0002:00000718* _ap_hack_apr_sdbm_unlock
0002:0000071c* _ap_hack_apr_sdbm_fetch
0002:00000720* _ap_hack_apr_sdbm_store
0002:00000724* _ap_hack_apr_sdbm_delete
0002:00000728* _ap_hack_apr_sdbm_firstkey
0002:0000072c* _ap_hack_apr_sdbm_nextkey
0002:00000730* _ap_hack_apr_sdbm_rdonly
0002:00000734* _ap_hack_apr_sha1_base64
0002:00000738* _ap_hack_apr_sha1_init
0002:0000073c* _ap_hack_apr_sha1_update
0002:00000740* _ap_hack_apr_sha1_update_binary
0002:00000744* _ap_hack_apr_sha1_final
0002:00000748* _ap_hack_apr_shm_create
0002:0000074c* _ap_hack_apr_shm_remove
0002:00000750* _ap_hack_apr_shm_destroy
0002:00000754* _ap_hack_apr_shm_attach
0002:00000758* _ap_hack_apr_shm_detach
0002:0000075c* _ap_hack_apr_shm_baseaddr_get
0002:00000760* _ap_hack_apr_shm_size_get
0002:00000764* _ap_hack_apr_shm_pool_get
0002:00000768* _ap_hack_apr_signal
0002:0000076c* _ap_hack_apr_signal_description_get
0002:00000770* _ap_hack_apr_signal_block
0002:00000774* _ap_hack_apr_signal_unblock
0002:00000778* _ap_hack_apr_strnatcmp
0002:0000077c* _ap_hack_apr_strnatcasecmp
0002:00000780* _ap_hack_apr_pstrdup
0002:00000784* _ap_hack_apr_pstrmemdup
0002:00000788* _ap_hack_apr_pstrndup
0002:0000078c* _ap_hack_apr_pmemdup
0002:00000790* _ap_hack_apr_pstrcat
0002:00000794* _ap_hack_apr_pstrcatv
0002:00000798* _ap_hack_apr_pvsprintf
0002:0000079c* _ap_hack_apr_psprintf
0002:000007a0* _ap_hack_apr_cpystrn
0002:000007a4* _ap_hack_apr_collapse_spaces
0002:000007a8* _ap_hack_apr_tokenize_to_argv
0002:000007ac* _ap_hack_apr_strtok
0002:000007b0* _ap_hack_apr_snprintf
0002:000007b4* _ap_hack_apr_vsnprintf
0002:000007b8* _ap_hack_apr_itoa
0002:000007bc* _ap_hack_apr_ltoa
0002:000007c0* _ap_hack_apr_off_t_toa
0002:000007c4* _ap_hack_apr_strtoff
0002:000007c8* _ap_hack_apr_strtoi64
0002:000007cc* _ap_hack_apr_atoi64
0002:000007d0* _ap_hack_apr_strfsize
0002:000007d4* _ap_hack_apr_strmatch_precompile
0002:000007d8* _ap_hack_apr_table_elts
0002:000007dc* _ap_hack_apr_is_empty_table
0002:000007e0* _ap_hack_apr_is_empty_array
0002:000007e4* _ap_hack_apr_array_make
0002:000007e8* _ap_hack_apr_array_push
0002:000007ec* _ap_hack_apr_array_pop
0002:000007f0* _ap_hack_apr_array_clear
0002:000007f4* _ap_hack_apr_array_cat
0002:000007f8* _ap_hack_apr_array_copy
0002:000007fc* _ap_hack_apr_array_copy_hdr
0002:00000800* _ap_hack_apr_array_append
0002:00000804* _ap_hack_apr_array_pstrcat
0002:00000808* _ap_hack_apr_table_make
0002:0000080c* _ap_hack_apr_table_copy
0002:00000810* _ap_hack_apr_table_clone
0002:00000814* _ap_hack_apr_table_clear
0002:00000818* _ap_hack_apr_table_get
0002:0000081c* _ap_hack_apr_table_set
0002:00000820* _ap_hack_apr_table_setn
0002:00000824* _ap_hack_apr_table_unset
0002:00000828* _ap_hack_apr_table_merge
0002:0000082c* _ap_hack_apr_table_mergen
0002:00000830* _ap_hack_apr_table_add
0002:00000834* _ap_hack_apr_table_addn
0002:00000838* _ap_hack_apr_table_overlay
0002:0000083c* _ap_hack_apr_table_do
0002:00000840* _ap_hack_apr_table_vdo
0002:00000844* _ap_hack_apr_table_overlap
0002:00000848* _ap_hack_apr_table_compress
0002:0000084c* _ap_hack_apr_thread_cond_create
0002:00000850* _ap_hack_apr_thread_cond_wait
0002:00000854* _ap_hack_apr_thread_cond_timedwait
0002:00000858* _ap_hack_apr_thread_cond_signal
0002:0000085c* _ap_hack_apr_thread_cond_broadcast
0002:00000860* _ap_hack_apr_thread_cond_destroy
0002:00000864* _ap_hack_apr_thread_cond_pool_get
0002:00000868* _ap_hack_apr_thread_mutex_create
0002:0000086c* _ap_hack_apr_thread_mutex_lock
0002:00000870* _ap_hack_apr_thread_mutex_trylock
0002:00000874* _ap_hack_apr_thread_mutex_unlock
0002:00000878* _ap_hack_apr_thread_mutex_destroy
0002:0000087c* _ap_hack_apr_thread_mutex_pool_get
0002:00000880* _ap_hack_apr_thread_pool_create
0002:00000884* _ap_hack_apr_thread_pool_destroy
0002:00000888* _ap_hack_apr_thread_pool_push
0002:0000088c* _ap_hack_apr_thread_pool_schedule
0002:00000890* _ap_hack_apr_thread_pool_top
0002:00000894* _ap_hack_apr_thread_pool_tasks_cancel
0002:00000898* _ap_hack_apr_thread_pool_tasks_count
0002:0000089c* _ap_hack_apr_thread_pool_scheduled_tasks_count
0002:000008a0* _ap_hack_apr_thread_pool_threads_count
0002:000008a4* _ap_hack_apr_thread_pool_busy_count
0002:000008a8* _ap_hack_apr_thread_pool_idle_count
0002:000008ac* _ap_hack_apr_thread_pool_idle_max_set
0002:000008b0* _ap_hack_apr_thread_pool_idle_max_get
0002:000008b4* _ap_hack_apr_thread_pool_thread_max_set
0002:000008b8* _ap_hack_apr_thread_pool_thread_max_get
0002:000008bc* _ap_hack_apr_thread_pool_threshold_set
0002:000008c0* _ap_hack_apr_thread_pool_threshold_get
0002:000008c4* _ap_hack_apr_thread_pool_task_owner_get
0002:000008c8* _ap_hack_apr_threadattr_create
0002:000008cc* _ap_hack_apr_threadattr_detach_set
0002:000008d0* _ap_hack_apr_threadattr_detach_get
0002:000008d4* _ap_hack_apr_threadattr_stacksize_set
0002:000008d8* _ap_hack_apr_threadattr_guardsize_set
0002:000008dc* _ap_hack_apr_thread_create
0002:000008e0* _ap_hack_apr_thread_exit
0002:000008e4* _ap_hack_apr_thread_join
0002:000008e8* _ap_hack_apr_thread_yield
0002:000008ec* _ap_hack_apr_thread_once_init
0002:000008f0* _ap_hack_apr_thread_once
0002:000008f4* _ap_hack_apr_thread_detach
0002:000008f8* _ap_hack_apr_thread_data_get
0002:000008fc* _ap_hack_apr_thread_data_set
0002:00000900* _ap_hack_apr_threadkey_private_create
0002:00000904* _ap_hack_apr_threadkey_private_get
0002:00000908* _ap_hack_apr_threadkey_private_set
0002:0000090c* _ap_hack_apr_threadkey_private_delete
0002:00000910* _ap_hack_apr_threadkey_data_get
0002:00000914* _ap_hack_apr_threadkey_data_set
0002:00000918* _ap_hack_apr_procattr_create
0002:0000091c* _ap_hack_apr_procattr_io_set
0002:00000920* _ap_hack_apr_procattr_child_in_set
0002:00000924* _ap_hack_apr_procattr_child_out_set
0002:00000928* _ap_hack_apr_procattr_child_err_set
0002:0000092c* _ap_hack_apr_procattr_dir_set
0002:00000930* _ap_hack_apr_procattr_cmdtype_set
0002:00000934* _ap_hack_apr_procattr_detach_set
0002:00000938* _ap_hack_apr_procattr_limit_set
0002:0000093c* _ap_hack_apr_procattr_child_errfn_set
0002:00000940* _ap_hack_apr_procattr_error_check_set
0002:00000944* _ap_hack_apr_procattr_addrspace_set
0002:00000948* _ap_hack_apr_procattr_user_set
0002:0000094c* _ap_hack_apr_procattr_group_set
0002:00000950* _ap_hack_apr_proc_fork
0002:00000954* _ap_hack_apr_proc_create
0002:00000958* _ap_hack_apr_proc_wait
0002:0000095c* _ap_hack_apr_proc_wait_all_procs
0002:00000960* _ap_hack_apr_proc_detach
0002:00000964* _ap_hack_apr_proc_other_child_register
0002:00000968* _ap_hack_apr_proc_other_child_unregister
0002:0000096c* _ap_hack_apr_proc_other_child_alert
0002:00000970* _ap_hack_apr_proc_other_child_refresh
0002:00000974* _ap_hack_apr_proc_other_child_refresh_all
0002:00000978* _ap_hack_apr_proc_kill
0002:0000097c* _ap_hack_apr_pool_note_subprocess
0002:00000980* _ap_hack_apr_thread_pool_get
0002:00000984* _ap_hack_apr_thread_rwlock_create
0002:00000988* _ap_hack_apr_thread_rwlock_rdlock
0002:0000098c* _ap_hack_apr_thread_rwlock_tryrdlock
0002:00000990* _ap_hack_apr_thread_rwlock_wrlock
0002:00000994* _ap_hack_apr_thread_rwlock_trywrlock
0002:00000998* _ap_hack_apr_thread_rwlock_unlock
0002:0000099c* _ap_hack_apr_thread_rwlock_destroy
0002:000009a0* _ap_hack_apr_thread_rwlock_pool_get
0002:000009a4* _ap_hack_apr_time_now
0002:000009a8* _ap_hack_apr_time_ansi_put
0002:000009ac* _ap_hack_apr_time_exp_tz
0002:000009b0* _ap_hack_apr_time_exp_gmt
0002:000009b4* _ap_hack_apr_time_exp_lt
0002:000009b8* _ap_hack_apr_time_exp_get
0002:000009bc* _ap_hack_apr_time_exp_gmt_get
0002:000009c0* _ap_hack_apr_sleep
0002:000009c4* _ap_hack_apr_rfc822_date
0002:000009c8* _ap_hack_apr_ctime
0002:000009cc* _ap_hack_apr_strftime
0002:000009d0* _ap_hack_apr_time_clock_hires
0002:000009d4* _ap_hack_apr_uri_port_of_scheme
0002:000009d8* _ap_hack_apr_uri_unparse
0002:000009dc* _ap_hack_apr_uri_parse
0002:000009e0* _ap_hack_apr_uri_parse_hostinfo
0002:000009e4* _ap_hack_apr_uid_current
0002:000009e8* _ap_hack_apr_uid_name_get
0002:000009ec* _ap_hack_apr_uid_get
0002:000009f0* _ap_hack_apr_uid_homepath_get
0002:000009f4* _ap_hack_apr_gid_name_get
0002:000009f8* _ap_hack_apr_gid_get
0002:000009fc* _ap_hack_apr_uuid_get
0002:00000a00* _ap_hack_apr_uuid_format
0002:00000a04* _ap_hack_apr_uuid_parse
0002:00000a08* _ap_hack_apr_version
0002:00000a0c* _ap_hack_apr_version_string
0002:00000a10* _ap_hack_apr_xlate_open
0002:00000a14* _ap_hack_apr_xlate_sb_get
0002:00000a18* _ap_hack_apr_xlate_conv_buffer
0002:00000a1c* _ap_hack_apr_xlate_conv_byte
0002:00000a20* _ap_hack_apr_xlate_close
0002:00000a24* _ap_hack_apr_text_append
0002:00000a28* _ap_hack_apr_xml_parser_create
0002:00000a2c* _ap_hack_apr_xml_parse_file
0002:00000a30* _ap_hack_apr_xml_parser_feed
0002:00000a34* _ap_hack_apr_xml_parser_done
0002:00000a38* _ap_hack_apr_xml_parser_geterror
0002:00000a3c* _ap_hack_apr_xml_to_text
0002:00000a40* _ap_hack_apr_xml_empty_elem
0002:00000a44* _ap_hack_apr_xml_quote_string
0002:00000a48* _ap_hack_apr_xml_quote_elem
0002:00000a4c* _ap_hack_apr_xml_insert_uri
0002:00000a50* _ap_hack_apu_version
0002:00000a54* _ap_hack_apu_version_string
0002:00000a58* _ap_hack_ap_listen_pre_config
0002:00000a5c* _ap_hack_ap_setup_listeners
0002:00000a60* _ap_hack_ap_close_listeners
0002:00000a64* _ap_hack_ap_set_listenbacklog
0002:00000a68* _ap_hack_ap_set_listener
0002:00000a6c* _ap_hack_ap_set_send_buffer_size
0002:00000a70* _ap_hack_ap_set_receive_buffer_size
0002:00000a74* _ap_hack_ap_mpm_run
0002:00000a78* _ap_hack_ap_graceful_stop_signalled
0002:00000a7c* _ap_hack_ap_os_create_privileged_process
0002:00000a80* _ap_hack_ap_mpm_query
0002:00000a84* _ap_hack_ap_register_provider
0002:00000a88* _ap_hack_ap_lookup_provider
0002:00000a8c* _ap_hack_ap_list_provider_names
0002:00000a90* _ap_hack_ap_regcomp
0002:00000a94* _ap_hack_ap_regexec
0002:00000a98* _ap_hack_ap_regerror
0002:00000a9c* _ap_hack_ap_regfree
0002:00000aa0* _ap_hack_ap_get_module_config
0002:00000aa4* _ap_hack_ap_set_module_config
0002:00000aa8* _ap_hack_ap_set_string_slot
0002:00000aac* _ap_hack_ap_set_int_slot
0002:00000ab0* _ap_hack_ap_method_is_limited
0002:00000ab4* _ap_hack_ap_set_string_slot_lower
0002:00000ab8* _ap_hack_ap_set_flag_slot
0002:00000abc* _ap_hack_ap_set_file_slot
0002:00000ac0* _ap_hack_ap_set_deprecated
0002:00000ac4* _ap_hack_ap_server_root_relative
0002:00000ac8* _ap_hack_ap_add_module
0002:00000acc* _ap_hack_ap_remove_module
0002:00000ad0* _ap_hack_ap_add_loaded_module
0002:00000ad4* _ap_hack_ap_remove_loaded_module
0002:00000ad8* _ap_hack_ap_find_module_name
0002:00000adc* _ap_hack_ap_find_linked_module
0002:00000ae0* _ap_hack_ap_pcfg_openfile
0002:00000ae4* _ap_hack_ap_pcfg_open_custom
0002:00000ae8* _ap_hack_ap_cfg_getline
0002:00000aec* _ap_hack_ap_cfg_getc
0002:00000af0* _ap_hack_ap_cfg_closefile
0002:00000af4* _ap_hack_ap_soak_end_container
0002:00000af8* _ap_hack_ap_build_cont_config
0002:00000afc* _ap_hack_ap_build_config
0002:00000b00* _ap_hack_ap_walk_config
0002:00000b04* _ap_hack_ap_check_cmd_context
0002:00000b08* _ap_hack_ap_single_module_configure
0002:00000b0c* _ap_hack_ap_setup_prelinked_modules
0002:00000b10* _ap_hack_ap_show_directives
0002:00000b14* _ap_hack_ap_show_modules
0002:00000b18* _ap_hack_ap_show_mpm
0002:00000b1c* _ap_hack_ap_read_config
0002:00000b20* _ap_hack_ap_run_rewrite_args
0002:00000b24* _ap_hack_ap_register_hooks
0002:00000b28* _ap_hack_ap_fixup_virtual_hosts
0002:00000b2c* _ap_hack_ap_create_request_config
0002:00000b30* _ap_hack_ap_create_per_dir_config
0002:00000b34* _ap_hack_ap_merge_per_dir_configs
0002:00000b38* _ap_hack_ap_create_conn_config
0002:00000b3c* _ap_hack_ap_parse_htaccess
0002:00000b40* _ap_hack_ap_init_virtual_host
0002:00000b44* _ap_hack_ap_process_resource_config
0002:00000b48* _ap_hack_ap_process_config_tree
0002:00000b4c* _ap_hack_ap_invoke_handler
0002:00000b50* _ap_hack_ap_find_command
0002:00000b54* _ap_hack_ap_find_command_in_modules
0002:00000b58* _ap_hack_ap_set_config_vectors
0002:00000b5c* _ap_hack_ap_hook_header_parser
0002:00000b60* _ap_hack_ap_hook_get_header_parser
0002:00000b64* _ap_hack_ap_run_header_parser
0002:00000b68* _ap_hack_ap_hook_pre_config
0002:00000b6c* _ap_hack_ap_hook_get_pre_config
0002:00000b70* _ap_hack_ap_run_pre_config
0002:00000b74* _ap_hack_ap_hook_test_config
0002:00000b78* _ap_hack_ap_hook_get_test_config
0002:00000b7c* _ap_hack_ap_run_test_config
0002:00000b80* _ap_hack_ap_hook_post_config
0002:00000b84* _ap_hack_ap_hook_get_post_config
0002:00000b88* _ap_hack_ap_run_post_config
0002:00000b8c* _ap_hack_ap_hook_open_logs
0002:00000b90* _ap_hack_ap_hook_get_open_logs
0002:00000b94* _ap_hack_ap_run_open_logs
0002:00000b98* _ap_hack_ap_hook_child_init
0002:00000b9c* _ap_hack_ap_hook_get_child_init
0002:00000ba0* _ap_hack_ap_run_child_init
0002:00000ba4* _ap_hack_ap_hook_handler
0002:00000ba8* _ap_hack_ap_hook_get_handler
0002:00000bac* _ap_hack_ap_run_handler
0002:00000bb0* _ap_hack_ap_hook_quick_handler
0002:00000bb4* _ap_hack_ap_hook_get_quick_handler
0002:00000bb8* _ap_hack_ap_run_quick_handler
0002:00000bbc* _ap_hack_ap_hook_optional_fn_retrieve
0002:00000bc0* _ap_hack_ap_hook_get_optional_fn_retrieve
0002:00000bc4* _ap_hack_ap_run_optional_fn_retrieve
0002:00000bc8* _ap_hack_ap_process_connection
0002:00000bcc* _ap_hack_ap_flush_conn
0002:00000bd0* _ap_hack_ap_lingering_close
0002:00000bd4* _ap_hack_ap_hook_create_connection
0002:00000bd8* _ap_hack_ap_hook_get_create_connection
0002:00000bdc* _ap_hack_ap_run_create_connection
0002:00000be0* _ap_hack_ap_hook_pre_connection
0002:00000be4* _ap_hack_ap_hook_get_pre_connection
0002:00000be8* _ap_hack_ap_run_pre_connection
0002:00000bec* _ap_hack_ap_hook_process_connection
0002:00000bf0* _ap_hack_ap_hook_get_process_connection
0002:00000bf4* _ap_hack_ap_run_process_connection
0002:00000bf8* _ap_hack_ap_bucket_eoc_make
0002:00000bfc* _ap_hack_ap_bucket_eoc_create
0002:00000c00* _ap_hack_ap_allow_options
0002:00000c04* _ap_hack_ap_allow_overrides
0002:00000c08* _ap_hack_ap_default_type
0002:00000c0c* _ap_hack_ap_document_root
0002:00000c10* _ap_hack_ap_get_remote_host
0002:00000c14* _ap_hack_ap_get_remote_logname
0002:00000c18* _ap_hack_ap_construct_url
0002:00000c1c* _ap_hack_ap_get_server_name
0002:00000c20* _ap_hack_ap_get_server_port
0002:00000c24* _ap_hack_ap_get_limit_req_body
0002:00000c28* _ap_hack_ap_get_limit_xml_body
0002:00000c2c* _ap_hack_ap_custom_response
0002:00000c30* _ap_hack_ap_is_recursion_limit_exceeded
0002:00000c34* _ap_hack_ap_exists_config_define
0002:00000c38* _ap_hack_ap_core_translate
0002:00000c3c* _ap_hack_ap_auth_type
0002:00000c40* _ap_hack_ap_auth_name
0002:00000c44* _ap_hack_ap_satisfies
0002:00000c48* _ap_hack_ap_requires
0002:00000c4c* _ap_hack_ap_register_request_note
0002:00000c50* _ap_hack_ap_get_request_note
0002:00000c54* _ap_hack_ap_add_per_dir_conf
0002:00000c58* _ap_hack_ap_add_per_url_conf
0002:00000c5c* _ap_hack_ap_add_file_conf
0002:00000c60* _ap_hack_ap_limit_section
0002:00000c64* _ap_hack_ap_get_server_protocol
0002:00000c68* _ap_hack_ap_set_server_protocol
0002:00000c6c* _ap_hack_ap_hook_get_mgmt_items
0002:00000c70* _ap_hack_ap_hook_get_get_mgmt_items
0002:00000c74* _ap_hack_ap_run_get_mgmt_items
0002:00000c78* _ap_hack_ap_open_stderr_log
0002:00000c7c* _ap_hack_ap_replace_stderr_log
0002:00000c80* _ap_hack_ap_log_error
0002:00000c84* _ap_hack_ap_log_perror
0002:00000c88* _ap_hack_ap_log_rerror
0002:00000c8c* _ap_hack_ap_log_cerror
0002:00000c90* _ap_hack_ap_error_log2stderr
0002:00000c94* _ap_hack_ap_log_pid
0002:00000c98* _ap_hack_ap_read_pid
0002:00000c9c* _ap_hack_ap_open_piped_log
0002:00000ca0* _ap_hack_ap_open_piped_log_ex
0002:00000ca4* _ap_hack_ap_close_piped_log
0002:00000ca8* _ap_hack_ap_hook_error_log
0002:00000cac* _ap_hack_ap_hook_get_error_log
0002:00000cb0* _ap_hack_ap_run_error_log
0002:00000cb4* _ap_hack_ap_hook_insert_error_filter
0002:00000cb8* _ap_hack_ap_hook_get_insert_error_filter
0002:00000cbc* _ap_hack_ap_run_insert_error_filter
0002:00000cc0* _ap_hack_ap_get_mime_headers
0002:00000cc4* _ap_hack_ap_get_mime_headers_core
0002:00000cc8* _ap_hack_ap_finalize_request_protocol
0002:00000ccc* _ap_hack_ap_send_error_response
0002:00000cd0* _ap_hack_ap_set_content_length
0002:00000cd4* _ap_hack_ap_set_keepalive
0002:00000cd8* _ap_hack_ap_rationalize_mtime
0002:00000cdc* _ap_hack_ap_make_content_type
0002:00000ce0* _ap_hack_ap_setup_make_content_type
0002:00000ce4* _ap_hack_ap_make_etag
0002:00000ce8* _ap_hack_ap_set_etag
0002:00000cec* _ap_hack_ap_set_last_modified
0002:00000cf0* _ap_hack_ap_meets_conditions
0002:00000cf4* _ap_hack_ap_send_fd
0002:00000cf8* _ap_hack_ap_method_register
0002:00000cfc* _ap_hack_ap_method_registry_init
0002:00000d00* _ap_hack_ap_make_method_list
0002:00000d04* _ap_hack_ap_copy_method_list
0002:00000d08* _ap_hack_ap_method_in_list
0002:00000d0c* _ap_hack_ap_method_list_add
0002:00000d10* _ap_hack_ap_method_list_remove
0002:00000d14* _ap_hack_ap_clear_method_list
0002:00000d18* _ap_hack_ap_set_content_type
0002:00000d1c* _ap_hack_ap_rputc
0002:00000d20* _ap_hack_ap_rputs
0002:00000d24* _ap_hack_ap_rwrite
0002:00000d28* _ap_hack_ap_rvputs
0002:00000d2c* _ap_hack_ap_vrprintf
0002:00000d30* _ap_hack_ap_rprintf
0002:00000d34* _ap_hack_ap_rflush
0002:00000d38* _ap_hack_ap_index_of_response
0002:00000d3c* _ap_hack_ap_get_status_line
0002:00000d40* _ap_hack_ap_setup_client_block
0002:00000d44* _ap_hack_ap_should_client_block
0002:00000d48* _ap_hack_ap_get_client_block
0002:00000d4c* _ap_hack_ap_discard_request_body
0002:00000d50* _ap_hack_ap_note_auth_failure
0002:00000d54* _ap_hack_ap_note_basic_auth_failure
0002:00000d58* _ap_hack_ap_note_digest_auth_failure
0002:00000d5c* _ap_hack_ap_get_basic_auth_pw
0002:00000d60* _ap_hack_ap_parse_uri
0002:00000d64* _ap_hack_ap_getline
0002:00000d68* _ap_hack_ap_rgetline_core
0002:00000d6c* _ap_hack_ap_method_number_of
0002:00000d70* _ap_hack_ap_method_name_of
0002:00000d74* _ap_hack_ap_hook_post_read_request
0002:00000d78* _ap_hack_ap_hook_get_post_read_request
0002:00000d7c* _ap_hack_ap_run_post_read_request
0002:00000d80* _ap_hack_ap_hook_log_transaction
0002:00000d84* _ap_hack_ap_hook_get_log_transaction
0002:00000d88* _ap_hack_ap_run_log_transaction
0002:00000d8c* _ap_hack_ap_hook_http_scheme
0002:00000d90* _ap_hack_ap_hook_get_http_scheme
0002:00000d94* _ap_hack_ap_run_http_scheme
0002:00000d98* _ap_hack_ap_hook_default_port
0002:00000d9c* _ap_hack_ap_hook_get_default_port
0002:00000da0* _ap_hack_ap_run_default_port
0002:00000da4* _ap_hack_ap_bucket_error_make
0002:00000da8* _ap_hack_ap_bucket_error_create
0002:00000dac* _ap_hack_ap_byterange_filter
0002:00000db0* _ap_hack_ap_http_header_filter
0002:00000db4* _ap_hack_ap_content_length_filter
0002:00000db8* _ap_hack_ap_old_write_filter
0002:00000dbc* _ap_hack_ap_set_sub_req_protocol
0002:00000dc0* _ap_hack_ap_finalize_sub_req_protocol
0002:00000dc4* _ap_hack_ap_send_interim_response
0002:00000dc8* _ap_hack_ap_process_request_internal
0002:00000dcc* _ap_hack_ap_sub_req_lookup_uri
0002:00000dd0* _ap_hack_ap_sub_req_lookup_file
0002:00000dd4* _ap_hack_ap_sub_req_lookup_dirent
0002:00000dd8* _ap_hack_ap_sub_req_method_uri
0002:00000ddc* _ap_hack_ap_sub_req_output_filter
0002:00000de0* _ap_hack_ap_run_sub_req
0002:00000de4* _ap_hack_ap_destroy_sub_req
0002:00000de8* _ap_hack_ap_internal_redirect
0002:00000dec* _ap_hack_ap_internal_redirect_handler
0002:00000df0* _ap_hack_ap_internal_fast_redirect
0002:00000df4* _ap_hack_ap_some_auth_required
0002:00000df8* _ap_hack_ap_is_initial_req
0002:00000dfc* _ap_hack_ap_update_mtime
0002:00000e00* _ap_hack_ap_allow_methods
0002:00000e04* _ap_hack_ap_allow_standard_methods
0002:00000e08* _ap_hack_ap_die
0002:00000e0c* _ap_hack_ap_hook_create_request
0002:00000e10* _ap_hack_ap_hook_get_create_request
0002:00000e14* _ap_hack_ap_run_create_request
0002:00000e18* _ap_hack_ap_hook_translate_name
0002:00000e1c* _ap_hack_ap_hook_get_translate_name
0002:00000e20* _ap_hack_ap_run_translate_name
0002:00000e24* _ap_hack_ap_hook_map_to_storage
0002:00000e28* _ap_hack_ap_hook_get_map_to_storage
0002:00000e2c* _ap_hack_ap_run_map_to_storage
0002:00000e30* _ap_hack_ap_hook_check_user_id
0002:00000e34* _ap_hack_ap_hook_get_check_user_id
0002:00000e38* _ap_hack_ap_run_check_user_id
0002:00000e3c* _ap_hack_ap_hook_fixups
0002:00000e40* _ap_hack_ap_hook_get_fixups
0002:00000e44* _ap_hack_ap_run_fixups
0002:00000e48* _ap_hack_ap_hook_type_checker
0002:00000e4c* _ap_hack_ap_hook_get_type_checker
0002:00000e50* _ap_hack_ap_run_type_checker
0002:00000e54* _ap_hack_ap_hook_access_checker
0002:00000e58* _ap_hack_ap_hook_get_access_checker
0002:00000e5c* _ap_hack_ap_run_access_checker
0002:00000e60* _ap_hack_ap_hook_auth_checker
0002:00000e64* _ap_hack_ap_hook_get_auth_checker
0002:00000e68* _ap_hack_ap_run_auth_checker
0002:00000e6c* _ap_hack_ap_hook_insert_filter
0002:00000e70* _ap_hack_ap_hook_get_insert_filter
0002:00000e74* _ap_hack_ap_run_insert_filter
0002:00000e78* _ap_hack_ap_location_walk
0002:00000e7c* _ap_hack_ap_directory_walk
0002:00000e80* _ap_hack_ap_file_walk
0002:00000e84* _ap_hack_ap_init_vhost_config
0002:00000e88* _ap_hack_ap_fini_vhost_config
0002:00000e8c* _ap_hack_ap_vhost_iterate_given_conn
0002:00000e90* _ap_hack_ap_update_vhost_given_ip
0002:00000e94* _ap_hack_ap_update_vhost_from_headers
0002:00000e98* _ap_hack_ap_matches_request_vhost
0002:00000e9c* _ap_hack_ap_get_server_revision
0002:00000ea0* _ap_hack_ap_get_server_version
0002:00000ea4* _ap_hack_ap_get_server_banner
0002:00000ea8* _ap_hack_ap_get_server_description
0002:00000eac* _ap_hack_ap_add_version_component
0002:00000eb0* _ap_hack_ap_get_server_built
0002:00000eb4* _ap_hack_ap_field_noparam
0002:00000eb8* _ap_hack_ap_ht_time
0002:00000ebc* _ap_hack_ap_getword
0002:00000ec0* _ap_hack_ap_getword_nc
0002:00000ec4* _ap_hack_ap_getword_white
0002:00000ec8* _ap_hack_ap_getword_white_nc
0002:00000ecc* _ap_hack_ap_getword_nulls
0002:00000ed0* _ap_hack_ap_getword_nulls_nc
0002:00000ed4* _ap_hack_ap_getword_conf
0002:00000ed8* _ap_hack_ap_getword_conf_nc
0002:00000edc* _ap_hack_ap_resolve_env
0002:00000ee0* _ap_hack_ap_size_list_item
0002:00000ee4* _ap_hack_ap_get_list_item
0002:00000ee8* _ap_hack_ap_find_list_item
0002:00000eec* _ap_hack_ap_get_token
0002:00000ef0* _ap_hack_ap_find_token
0002:00000ef4* _ap_hack_ap_find_last_token
0002:00000ef8* _ap_hack_ap_is_url
0002:00000efc* _ap_hack_ap_unescape_url
0002:00000f00* _ap_hack_ap_unescape_url_keep2f
0002:00000f04* _ap_hack_ap_no2slash
0002:00000f08* _ap_hack_ap_getparents
0002:00000f0c* _ap_hack_ap_escape_path_segment
0002:00000f10* _ap_hack_ap_os_escape_path
0002:00000f14* _ap_hack_ap_escape_html
0002:00000f18* _ap_hack_ap_escape_html2
0002:00000f1c* _ap_hack_ap_escape_logitem
0002:00000f20* _ap_hack_ap_escape_errorlog_item
0002:00000f24* _ap_hack_ap_construct_server
0002:00000f28* _ap_hack_ap_escape_shell_cmd
0002:00000f2c* _ap_hack_ap_count_dirs
0002:00000f30* _ap_hack_ap_make_dirstr_prefix
0002:00000f34* _ap_hack_ap_make_dirstr_parent
0002:00000f38* _ap_hack_ap_make_full_path
0002:00000f3c* _ap_hack_ap_os_is_path_absolute
0002:00000f40* _ap_hack_ap_is_matchexp
0002:00000f44* _ap_hack_ap_strcmp_match
0002:00000f48* _ap_hack_ap_strcasecmp_match
0002:00000f4c* _ap_hack_ap_strcasestr
0002:00000f50* _ap_hack_ap_stripprefix
0002:00000f54* _ap_hack_ap_pbase64decode
0002:00000f58* _ap_hack_ap_pbase64encode
0002:00000f5c* _ap_hack_ap_pregcomp
0002:00000f60* _ap_hack_ap_pregfree
0002:00000f64* _ap_hack_ap_pregsub
0002:00000f68* _ap_hack_ap_content_type_tolower
0002:00000f6c* _ap_hack_ap_str_tolower
0002:00000f70* _ap_hack_ap_ind
0002:00000f74* _ap_hack_ap_rind
0002:00000f78* _ap_hack_ap_escape_quotes
0002:00000f7c* _ap_hack_ap_append_pid
0002:00000f80* _ap_hack_ap_timeout_parameter_parse
0002:00000f84* _ap_hack_ap_is_rdirectory
0002:00000f88* _ap_hack_ap_is_directory
0002:00000f8c* _ap_hack_ap_log_assert
0002:00000f90* _ap_hack_ap_psignature
0002:00000f94* _ap_hack_ap_strchr
0002:00000f98* _ap_hack_ap_strchr_c
0002:00000f9c* _ap_hack_ap_strrchr
0002:00000fa0* _ap_hack_ap_strrchr_c
0002:00000fa4* _ap_hack_ap_strstr
0002:00000fa8* _ap_hack_ap_strstr_c
0002:00000fac* _ap_hack_ap_uname2id
0002:00000fb0* _ap_hack_ap_gname2id
0002:00000fb4* _ap_hack_ap_hook_monitor
0002:00000fb8* _ap_hack_ap_hook_get_monitor
0002:00000fbc* _ap_hack_ap_run_monitor
0002:00000fc0* _ap_hack_ap_exists_scoreboard_image
0002:00000fc4* _ap_hack_ap_increment_counts
0002:00000fc8* _ap_hack_ap_calc_scoreboard_size
0002:00000fcc* _ap_hack_ap_create_sb_handle
0002:00000fd0* _ap_hack_ap_update_child_status
0002:00000fd4* _ap_hack_ap_update_child_status_from_indexes
0002:00000fd8* _ap_hack_ap_get_scoreboard_worker
0002:00000fdc* _ap_hack_ap_get_scoreboard_process
0002:00000fe0* _ap_hack_ap_get_scoreboard_global
0002:00000fe4* _ap_hack_ap_get_scoreboard_lb
0002:00000fe8* _ap_hack_ap_hook_pre_mpm
0002:00000fec* _ap_hack_ap_hook_get_pre_mpm
0002:00000ff0* _ap_hack_ap_run_pre_mpm
0002:00000ff4* _ap_hack_ap_get_brigade
0002:00000ff8* _ap_hack_ap_pass_brigade
0002:00000ffc* _ap_hack_ap_register_input_filter
0002:00001000* _ap_hack_ap_register_output_filter
0002:00001004* _ap_hack_ap_register_output_filter_protocol
0002:00001008* _ap_hack_ap_add_input_filter
0002:0000100c* _ap_hack_ap_add_input_filter_handle
0002:00001010* _ap_hack_ap_get_input_filter_handle
0002:00001014* _ap_hack_ap_add_output_filter
0002:00001018* _ap_hack_ap_add_output_filter_handle
0002:0000101c* _ap_hack_ap_get_output_filter_handle
0002:00001020* _ap_hack_ap_remove_input_filter
0002:00001024* _ap_hack_ap_remove_output_filter
0002:00001028* _ap_hack_ap_save_brigade
0002:0000102c* _ap_hack_ap_filter_flush
0002:00001030* _ap_hack_ap_fflush
0002:00001034* _ap_hack_ap_fputstrs
0002:00001038* _ap_hack_ap_fprintf
0002:0000103c* _ap_hack_ap_filter_protocol
0002:00001040* _ap_hack_ap_md5
0002:00001044* _ap_hack_ap_md5_binary
0002:00001048* _ap_hack_ap_md5contextTo64
0002:0000104c* _ap_hack_ap_md5digest
0002:00001050* _ap_hack_ap_create_environment
0002:00001054* _ap_hack_ap_find_path_info
0002:00001058* _ap_hack_ap_add_cgi_vars
0002:0000105c* _ap_hack_ap_add_common_vars
0002:00001060* _ap_hack_ap_scan_script_header_err
0002:00001064* _ap_hack_ap_scan_script_header_err_brigade
0002:00001068* _ap_hack_ap_scan_script_header_err_strs
0002:0000106c* _ap_hack_ap_scan_script_header_err_core
0002:00001070* _ap_hack_ap_explode_recent_localtime
0002:00001074* _ap_hack_ap_explode_recent_gmt
0002:00001078* _ap_hack_ap_recent_ctime
0002:0000107c* _ap_hack_ap_recent_rfc822_date
0002:00001080* _ap_hack_ap_xml_parse_input
0002:00001084* _ap_hack_ap_basic_http_header
0002:00001088* _ap_hack_ap_send_http_trace
0002:0000108c* _ap_hack_ap_send_http_options
0002:00002bd0  _ap_ugly_hack
Module: U:\dev\httpd-2.2.17\modules.o(modules.o)
0002:00001090  _ap_prelinked_modules
0002:000010b0  _ap_prelinked_module_symbols
0002:000010e0  _ap_preloaded_modules
Module: U:\dev\httpd-2.2.17\server\.libs\main.lib(main.o)
0001:00000110* _suck_in_APR
0001:00000fe4  _main
0001:00000fe4* main
Module: U:\usr\lib\tcpipv4\libc_dll.lib(swapl.obj)
0001:00001f90  __swapl
Module: U:\extras\lib\apr-1.lib(apr_pools.o)
0001:00001fa0  _apr_allocator_mutex_set
0001:00001fb0  _apr_allocator_mutex_get
0001:00001fbc  _apr_allocator_owner_set
0001:00001fcc  _apr_allocator_owner_get
0001:00001fd8  _apr_pool_abort_set
0001:00001fe8  _apr_pool_abort_get
0001:00001ff4  _apr_pool_parent_get
0001:00002000  _apr_pool_allocator_get
0001:0000200c  _apr_pool_is_ancestor
0001:00002038  _apr_pool_tag
0001:00002048  _apr_pool_cleanup_kill
0001:000020bc  _apr_pool_child_cleanup_set
0001:000020f4  _apr_pool_cleanup_run
0001:00002124  _apr_pool_cleanup_for_exec
0001:0000212c  _apr_pool_cleanup_null
0001:00002134  _apr_pool_userdata_get
0001:0000217c  _apr_allocator_max_free_set
0001:000021d4  _apr_allocator_destroy
0001:00002534  _apr_pvsprintf
0001:00002764  _apr_psprintf
0001:00002788  _apr_allocator_create
0001:000029b4  _apr_allocator_free
0001:00002a94  _apr_pool_destroy
0001:00002c5c  _apr_pool_destroy_debug
0001:00002c68  _apr_pool_terminate
0001:00002ca8  _apr_pool_clear
0001:00002e38  _apr_pool_clear_debug
0001:00002e44  _apr_allocator_alloc
0001:00002fdc  _apr_pool_create_ex
0001:00003288  _apr_pool_create_ex_debug
0001:000032a4  _apr_pool_initialize
0001:0000337c  _apr_pool_create_unmanaged_ex
0001:000035d0  _apr_pool_create_unmanaged_ex_debug
0001:000035dc  _apr_pool_create_core_ex_debug
0001:000035e8  _apr_pool_create_core_ex
0001:000035f4  _apr_palloc
0001:0000397c  _apr_palloc_debug
0001:00003988  _apr_pool_note_subprocess
0001:000039bc  _apr_pool_pre_cleanup_register
0001:00003a04  _apr_pool_cleanup_register
0001:00003a54  _apr_pool_userdata_setn
0001:00003abc  _apr_pool_userdata_set
0001:00003b70* _apr_pcalloc
0001:00003ba4  _apr_pcalloc_debug
Module: U:\extras\lib\apr-1.lib(ia32.o)
0001:00003bb0  _apr_atomic_init
0001:00003bb8  _apr_atomic_read32
0001:00003bc4  _apr_atomic_set32
0001:00003bd4  _apr_atomic_add32
0001:00003be4  _apr_atomic_sub32
0001:00003bf4  _apr_atomic_inc32
0001:00003c08  _apr_atomic_dec32
0001:00003c1c  _apr_atomic_cas32
0001:00003c30  _apr_atomic_xchg32
0001:00003c40  _apr_atomic_casptr
0001:00003c54  _apr_atomic_xchgptr
Module: U:\extras\lib\aprutil-1.lib(apr_base64.o)
0001:00003c70  _apr_base64_decode_len
0001:00003ca4  _apr_base64_decode_binary
0001:00003e04  _apr_base64_decode
0001:00003e28  _apr_base64_encode_len
0001:00003e48  _apr_base64_encode_binary
0001:00003f74  _apr_base64_encode
Module: U:\extras\lib\aprutil-1.lib(apr_brigade.o)
0001:000040d0  _apr_brigade_cleanup
0001:00004128  _apr_brigade_partition
0001:000042e4  _apr_brigade_length
0001:00004390  _apr_brigade_to_iovec
0001:0000441c  _apr_brigade_insert_file
0001:000045a8  _apr_brigade_flatten
0001:00004640  _apr_brigade_writev
0001:000048e0  _apr_brigade_write
0001:00004a44  _apr_brigade_vprintf
0001:00004ac8  _apr_brigade_printf
0001:00004b50  _apr_brigade_puts
0001:00004bdc  _apr_brigade_putc
0001:00004c14  _apr_brigade_vputstrs
0001:00004c74  _apr_brigade_putstrs
0001:00004c9c  _apr_brigade_split_line
0001:00004e34  _apr_brigade_pflatten
0001:00004e94  _apr_brigade_create
0001:00004ee8  _apr_brigade_split_ex
0001:00004f60  _apr_brigade_split
0001:00004f84  _apr_brigade_destroy
Module: U:\extras\lib\aprutil-1.lib(apr_buckets_alloc.o)
0001:00004fc0  _apr_bucket_free
0001:00005018  _apr_bucket_alloc
0001:000050b4  _apr_bucket_alloc_create_ex
0001:00005100  _apr_bucket_alloc_destroy
0001:0000513c  _apr_bucket_alloc_create
Module: U:\extras\lib\aprutil-1.lib(apr_buckets.o)
0001:00005180  _apr_bucket_setaside_noop
0001:00005188  _apr_bucket_setaside_notimpl
0001:00005194  _apr_bucket_split_notimpl
0001:000051a0  _apr_bucket_copy_notimpl
0001:000051ac  _apr_bucket_destroy_noop
Module: U:\extras\lib\aprutil-1.lib(apr_buckets_simple.o)
0001:000051e0  _apr_bucket_immortal_make
0001:000053b0  _apr_bucket_type_immortal
0001:0000520c  _apr_bucket_transient_make
0001:000053e0  _apr_bucket_type_transient
0001:0000526c  _apr_bucket_transient_create
0001:000052bc  _apr_bucket_immortal_create
0001:0000530c  _apr_bucket_simple_copy
0001:00005344  _apr_bucket_simple_split
Module: U:\extras\lib\aprutil-1.lib(apr_buckets_refcount.o)
0001:00005400  _apr_bucket_shared_destroy
0001:00005418  _apr_bucket_shared_make
0001:00005440  _apr_bucket_shared_copy
0001:00005468  _apr_bucket_shared_split
Module: U:\extras\lib\aprutil-1.lib(apr_buckets_eos.o)
0001:000054ac  _apr_bucket_eos_make
0001:00005530  _apr_bucket_type_eos
0001:000054d8  _apr_bucket_eos_create
Module: U:\extras\lib\aprutil-1.lib(apr_buckets_flush.o)
0001:0000556c  _apr_bucket_flush_make
0001:000055f0  _apr_bucket_type_flush
0001:00005598  _apr_bucket_flush_create
Module: U:\extras\lib\aprutil-1.lib(apr_buckets_heap.o)
0001:00005664  _apr_bucket_heap_make
0001:00005770  _apr_bucket_type_heap
0001:00005718  _apr_bucket_heap_create
Module: U:\extras\lib\aprutil-1.lib(apr_buckets_pool.o)
0001:00005860  _apr_bucket_pool_make
0001:00005960  _apr_bucket_type_pool
0001:000058fc  _apr_bucket_pool_create
Module: U:\extras\lib\aprutil-1.lib(apr_buckets_socket.o)
0001:00005980  _apr_bucket_socket_make
0001:00005bb0  _apr_bucket_type_socket
0001:000059ac  _apr_bucket_socket_create
Module: U:\extras\lib\aprutil-1.lib(apr_buckets_pipe.o)
0001:00005bd0  _apr_bucket_pipe_make
0001:00005e10  _apr_bucket_type_pipe
0001:00005bfc  _apr_bucket_pipe_create
Module: U:\extras\lib\aprutil-1.lib(apr_buckets_file.o)
0001:00005e30  _apr_bucket_file_enable_mmap
0001:000061b0  _apr_bucket_type_file
0001:000060d8  _apr_bucket_file_make
0001:00006134  _apr_bucket_file_create
Module: U:\extras\lib\aprutil-1.lib(apr_date.o)
0001:000061d0  _apr_date_checkmask
0001:000063c0  _apr_date_parse_rfc
0001:00006bf4  _apr_date_parse_http
Module: U:\extras\lib\aprutil-1.lib(apr_dbd.o)
0001:00006fe4  _apr_dbd_open_ex
0001:0000706c  _apr_dbd_open
0001:0000709c  _apr_dbd_transaction_mode_get
0001:000070b4  _apr_dbd_transaction_mode_set
0001:000070d0  _apr_dbd_close
0001:000070e8  _apr_dbd_name
0001:000070f4  _apr_dbd_native_handle
0001:0000710c  _apr_dbd_check_conn
0001:00007128  _apr_dbd_set_dbname
0001:0000714c  _apr_dbd_query
0001:00007170  _apr_dbd_select
0001:000071a8  _apr_dbd_num_cols
0001:000071c0  _apr_dbd_num_tuples
0001:000071d8  _apr_dbd_get_row
0001:00007200  _apr_dbd_get_entry
0001:0000721c  _apr_dbd_get_name
0001:00007238  _apr_dbd_error
0001:00007254  _apr_dbd_escape
0001:00007278  _apr_dbd_pquery
0001:000072b0  _apr_dbd_pselect
0001:000072ec  _apr_dbd_pbquery
0001:00007324  _apr_dbd_pbselect
0001:00007360  _apr_dbd_datum_get
0001:00007388  _apr_dbd_pvbselect
0001:000073c0  _apr_dbd_pvbquery
0001:000073f0  _apr_dbd_pvselect
0001:00007428  _apr_dbd_pvquery
0001:00007458  _apr_dbd_prepare
0001:000078f4  _apr_dbd_transaction_end
0001:00007928  _apr_dbd_transaction_start
0001:0000799c  _apr_dbd_get_driver
0001:00007af0  _apr_dbd_init
0001:00007bb8* _apr_dbd_mutex_unlock
0001:00007bd0* _apr_dbd_mutex_lock
Module: U:\extras\lib\aprutil-1.lib(apr_dbm.o)
0001:00007c04  _apr_dbm_close
0001:00007c18  _apr_dbm_fetch
0001:00007c30  _apr_dbm_store
0001:00007c48  _apr_dbm_delete
0001:00007c5c  _apr_dbm_exists
0001:00007c70  _apr_dbm_firstkey
0001:00007c84  _apr_dbm_nextkey
0001:00007c98  _apr_dbm_freedatum
0001:00007cac* _apr_posix_perms2mode
0001:00007ff8  _apr_dbm_get_usednames_ex
0001:00008048  _apr_dbm_get_usednames
0001:00008078  _apr_dbm_open_ex
0001:000080d0  _apr_dbm_open
0001:00008108  _apr_dbm_geterror
Module: U:\extras\lib\apr-1.lib(dso.o)
0001:00008150  _apr_os_dso_handle_get
0001:00008164  _apr_os_dso_handle_put
0001:000081a4  _apr_dso_error
0001:0000823c  _apr_dso_sym
0001:000082e8  _apr_dso_unload
0001:0000834c  _apr_dso_load
Module: U:\extras\lib\apr-1.lib(env.o)
0001:00008440  _apr_env_delete
0001:00008458  _apr_env_set
0001:00008480  _apr_env_get
Module: U:\extras\lib\apr-1.lib(errorcodes.o)
0001:00008db8  _apr_strerror
Module: U:\extras\lib\apr-1.lib(filestat.o)
0001:000091e0  _apr_file_perms_set
0001:000091ec  _apr_file_mtime_set
0001:00009284  _apr_file_attrs_set
0001:00009428  _apr_stat
0001:00009560  _apr_file_info_get
0001:000096a4  _apr_file_info_get_locked
Module: U:\extras\lib\apr-1.lib(dir.o)
0001:00009860  _apr_os_dir_get
0001:00009880  _apr_os_dir_put
0001:000098cc  _apr_dir_remove
0001:000098f8  _apr_dir_make
0001:00009934  _apr_dir_read
0001:00009abc  _apr_dir_close
0001:00009afc  _apr_dir_rewind
0001:00009b14  _apr_dir_open
Module: U:\extras\lib\apr-1.lib(filepath.o)
0001:00009bc0  _apr_filepath_encoding
0001:00009bd0  _apr_filepath_list_merge
0001:00009bfc  _apr_filepath_list_split
0001:00009c28  _apr_filepath_root
0001:00009fc4  _apr_filepath_merge
Module: U:\extras\lib\apr-1.lib(filesys.o)
0001:0000acd0  _filepath_root_test
0001:0000ad08  _apr_filepath_set
0001:0000ad50  _apr_filepath_get
0001:0000adf0  _filepath_root_case
0001:0000ae50  _filepath_drive_get
0001:0000af10  _c_is_fnchar
Module: U:\extras\lib\apr-1.lib(open.o)
0001:0000b010  _apr_os_file_get
0001:0000b024  _apr_file_eof
0001:0000b044  _apr_file_pool_get
0001:0000b050  _apr_file_link
0001:0000b05c  _apr_file_inherit_unset
0001:0000b084  _apr_file_inherit_set
0001:0000b0d8  _apr_os_file_put
0001:0000b184  _apr_file_open_flags_stdin
0001:0000b1b8  _apr_file_open_stdin
0001:0000b1dc  _apr_file_open_flags_stdout
0001:0000b210  _apr_file_open_stdout
0001:0000b234  _apr_file_open_flags_stderr
0001:0000b268  _apr_file_open_stderr
0001:0000b28c  _apr_file_rename
0001:0000b2e4  _apr_file_remove
0001:0000b300  _apr_file_close
0001:0000b37c  _apr_file_cleanup
0001:0000b388  _apr_file_open
0001:0000b714  _apr_unix_child_file_cleanup
0001:0000b720  _apr_unix_file_cleanup
Module: U:\extras\lib\apr-1.lib(copy.o)
0001:0000b90c  _apr_file_append
0001:0000b93c  _apr_file_copy
Module: U:\extras\lib\apr-1.lib(readwrite.o)
0001:0000b970  _apr_file_sync
0001:0000b97c  _apr_file_datasync
0001:0000b988* _apr_file_check_read
0001:0000ba18  _apr_file_printf
0001:0000ba98  _apr_file_flush
0001:0000bb04  _apr_file_putc
0001:0000bb50  _apr_file_flush_locked
0001:0000bbbc  _apr_file_puts
0001:0000bbf8  _apr_file_ungetc
0001:0000bc28  _apr_file_writev
0001:0000bd0c  _apr_file_write
0001:0000bf58  _apr_file_read
0001:0000c22c  _apr_file_gets
0001:0000c2cc  _apr_file_getc
Module: U:\extras\lib\apr-1.lib(fullrw.o)
0001:0000c300  _apr_file_write_full
0001:0000c350  _apr_file_writev_full
0001:0000c4e4  _apr_file_read_full
Module: U:\extras\lib\apr-1.lib(filedup.o)
0001:0000c540  _apr_file_setaside
0001:0000c748  _apr_file_dup2
0001:0000c76c  _apr_file_dup
Module: U:\extras\lib\apr-1.lib(buffer.o)
0001:0000c7b0  _apr_file_buffer_size_get
0001:0000c7bc  _apr_file_buffer_set
Module: U:\extras\lib\apr-1.lib(seek.o)
0001:0000c8e8  _apr_file_trunc
0001:0000c93c  _apr_file_seek
Module: U:\extras\lib\apr-1.lib(pipe.o)
0001:0000ca80  _apr_file_namedpipe_create
0001:0000ca8c  _apr_file_pipe_timeout_get
0001:0000cab4  _apr_os_pipe_put_ex
0001:0000cb34  _apr_os_pipe_put
0001:0000cb60  _apr_file_pipe_timeout_set
0001:0000cbe8  _apr_file_pipe_create
0001:0000cf30  _apr_file_pipe_create_ex
Module: U:\extras\lib\apr-1.lib(flock.o)
0001:0000cfe0  _apr_file_unlock
0001:0000d02c  _apr_file_lock
Module: U:\extras\lib\apr-1.lib(fileacc.o)
0001:0000d090  _apr_file_name_get
0001:0000d0a4  _apr_file_flags_get
0001:0000d0b0* _apr_unix_perms2mode
0001:0000d124  _apr_unix_mode2perms
0001:0000d198  _apr_file_data_set
0001:0000d1c4  _apr_file_data_get
Module: U:\extras\lib\apr-1.lib(dir_make_recurse.o)
0001:0000d1e0  _apr_dir_make_recursive
Module: U:\extras\lib\apr-1.lib(mktemp.o)
0001:0000d340  _apr_file_mktemp
Module: U:\extras\lib\apr-1.lib(tempdir.o)
0001:0000d4c0  _apr_temp_dir_get
Module: U:\extras\lib\apr-1.lib(apr_fnmatch.o)
0001:0000d640  _apr_fnmatch_test
0001:0000d68c  _apr_fnmatch
0001:0000da48  _apr_match_glob
Module: U:\extras\lib\apr-1.lib(start.o)
0001:0000db70  _apr_terminate
0001:0000db90  _apr_terminate2
0001:0000dba8  _apr_initialize
0001:0000dc2c  _apr_app_initialize
Module: U:\extras\lib\apr-1.lib(rand.o)
0001:0000dc40* _randbyte
0001:0000dc5c  _apr_generate_random_bytes
Module: U:\extras\lib\apr-1.lib(getopt.o)
0001:0000de2c  _apr_getopt_long
0001:0000e1c0  _apr_getopt
0001:0000e3b4  _apr_getopt_init
Module: U:\extras\lib\apr-1.lib(apr_hash.o)
0001:0000e460  _apr_hash_next
0001:0000e4b4  _apr_hash_this
0001:0000e4f0  _apr_hashfunc_default
0001:0000e55c  _apr_hash_count
0001:0000e568  _apr_hash_do
0001:0000e618  _apr_hash_pool_get
0001:0000e624  _apr_hash_copy
0001:0000e6e8  _apr_hash_first
0001:0000e838  _apr_hash_get
0001:0000e8a4  _apr_hash_merge
0001:0000eaf8  _apr_hash_overlay
0001:0000eb2c  _apr_hash_set
0001:0000ec20  _apr_hash_clear
0001:0000ecac  _apr_hash_make
0001:0000ed04  _apr_hash_make_custom
Module: U:\extras\lib\aprutil-1.lib(apr_hooks.o)
0001:0000ed34  _apr_hook_deregister_all
0001:0000ed7c  _apr_dynamic_fn_register
0001:0000edd8  _apr_dynamic_fn_retrieve
0001:0000ee20  _apr_optional_hook_get
0001:0000ee6c  _apr_hook_sort_register
0001:0000eed0  _apr_hook_debug_show
0001:0000effc  _apr_optional_hook_add
0001:0000f164  _apr_hook_sort_all
0002:00002c80  _apr_hook_global_pool
0002:00002c88  _apr_hook_debug_current
0002:00002c84  _apr_hook_debug_enabled
0002:00002c8c* _apr_global_hook_pool
0002:00002c90* _apr_debug_module_hooks
0002:00002c94* _apr_current_hooking_module
Module: U:\extras\lib\apr-1.lib(apr_cpystrn.o)
0001:0000f6a0  _apr_cpystrn
0001:0000f6d8  _apr_collapse_spaces
0001:0000f708  _apr_filepath_name_get
0001:0000f738  _apr_tokenize_to_argv
Module: U:\extras\lib\apr-1.lib(apr_snprintf.o)
0001:0000fe34  _apr_vformatter
0001:000117a0  _apr_vsnprintf
0001:00011820  _apr_snprintf
Module: U:\extras\lib\apr-1.lib(apr_getpass.o)
0001:00011940  _apr_password_get
Module: U:\extras\lib\aprutil-1.lib(apr_md4.o)
0001:000119c0  _apr_md4_init
0001:00011efc  _apr_md4_update
0001:000120c4  _apr_md4_final
0001:0001219c  _apr_md4
0001:00012208  _apr_md4_set_xlate
Module: U:\extras\lib\aprutil-1.lib(apr_md5.o)
0001:00012240  _apr_md5_init
0001:00012bc0  _apr_md5_update
0001:00012bec  _apr_md5_final
0001:00012cc4  _apr_md5
0001:00012d30  _apr_md5_encode
0001:00013360  _apr_password_validate
0001:00013448  _apr_md5_set_xlate
Module: U:\extras\lib\aprutil-1.lib(apr_memcache.o)
0001:00013520  _apr_memcache_add_server
0001:0001355c  _apr_memcache_enable_server
0001:00013574  _apr_memcache_hash_crc32
0001:000135b0  _apr_memcache_hash_default
0001:000135f4  _apr_memcache_hash
0001:00013650  _apr_memcache_create
0001:00013a24  _apr_memcache_stats
0001:0001405c  _apr_memcache_version
0001:00014164  _apr_memcache_add_multget_key
0001:000141f4  _apr_memcache_find_server
0001:0001424c  _apr_memcache_server_create
0001:00014584  _apr_memcache_disable_server
0001:00014694  _apr_memcache_find_server_hash_default
0001:0001482c  _apr_memcache_find_server_hash
0001:00014878  _apr_memcache_multgetp
0001:00015168  _apr_memcache_delete
0001:00015330  _apr_memcache_getp
0001:00015844  _apr_memcache_replace
0001:00015890  _apr_memcache_add
0001:000158dc  _apr_memcache_set
0001:00015b14  _apr_memcache_incr
0001:00015b4c  _apr_memcache_decr
Module: U:\extras\lib\apr-1.lib(sockets.o)
0001:00015fe4  _apr_socket_protocol_get
0001:00015ff8  _apr_socket_shutdown
0001:00016034  _apr_socket_bind
0001:000160a0  _apr_socket_listen
0001:000160dc  _apr_socket_connect
0001:0001615c  _apr_socket_type_get
0001:00016170  _apr_os_sock_get
0001:00016184  _apr_socket_pool_get
0001:00016190  _apr_socket_inherit_set
0001:0001619c  _apr_socket_inherit_unset
0001:000162ac  _apr_os_sock_put
0001:00016334  _apr_os_sock_make
0001:0001641c  _apr_socket_accept
0001:00016524  _apr_socket_create
0001:000165ec  _apr_socket_data_set
0001:00016658  _apr_socket_data_get
0001:000166a4  _apr_socket_close
Module: U:\extras\lib\apr-1.lib(socket_util.o)
0001:000166e0  _apr_socket_atreadeof
Module: U:\extras\lib\apr-1.lib(sockaddr.o)
0001:000167e0  _apr_sockaddr_vars_set
0001:00016828  _apr_ipsubnet_test
0001:00016844  _apr_ipsubnet_create
0001:00016ae8  _apr_sockaddr_equal
0001:00016b18  _apr_getservbyname
0001:00016b8c  _apr_getnameinfo
0001:00016c00  _apr_sockaddr_info_get
0001:00016e08  _apr_parse_addr_port
0001:00016ef8  _apr_socket_addr_get
0001:0001701c  _apr_sockaddr_ip_getbuf
0001:00017068  _apr_sockaddr_ip_get
Module: U:\extras\lib\apr-1.lib(sockopt.o)
0001:000170b0  _apr_socket_timeout_set
0001:000170c8  _apr_socket_opt_set
0001:000172dc  _apr_socket_timeout_get
0001:000172f4  _apr_socket_opt_get
0001:00017504  _apr_socket_atmark
0001:00017560  _apr_gethostname
Module: U:\extras\lib\apr-1.lib(sendrecv.o)
0001:000175d0  _apr_socket_send
0001:00017704  _apr_socket_recv
0001:0001786c  _apr_socket_sendv
Module: U:\extras\lib\apr-1.lib(sendrecv_udp.o)
0001:000179e0  _apr_socket_sendto
0001:00017afc  _apr_socket_recvfrom
Module: U:\extras\lib\apr-1.lib(pollset.o)
0001:00017c50  _apr_pollset_destroy
0001:00017c58  _apr_pollset_add
0001:00017cb0  _apr_pollset_remove
0001:00017da0  _apr_pollset_poll
0001:0001807c  _apr_pollset_create
0001:00018108  _apr_pollset_create_ex
Module: U:\extras\lib\apr-1.lib(poll.o)
0001:00018120  _apr_pollcb_create
0001:0001812c  _apr_pollcb_add
0001:00018138  _apr_pollcb_remove
0001:00018144  _apr_pollcb_poll
0001:00018150  _apr_poll
Module: U:\extras\lib\apr-1.lib(proc_mutex.o)
0001:000183e0  _apr_proc_mutex_lockfile
0001:000183f0  _apr_proc_mutex_name
0001:000183fc  _apr_proc_mutex_defname
0001:00018408  _apr_proc_mutex_pool_get
0001:00018414  _apr_os_proc_mutex_get
0001:0001842c  _apr_os_proc_mutex_put
0001:0001846c  _apr_proc_mutex_unlock
0001:000184b4  _apr_proc_mutex_destroy
0001:00018530  _apr_proc_mutex_cleanup
0001:0001853c  _apr_proc_mutex_trylock
0001:00018580  _apr_proc_mutex_lock
0001:000185cc  _apr_proc_mutex_child_init
0001:0001868c  _apr_proc_mutex_create
Module: U:\extras\lib\apr-1.lib(time.o)
0001:00018770  _apr_time_ansi_put
0001:00018790  _apr_time_exp_get
0001:000189a0  _apr_time_exp_gmt_get
0001:000189dc  _apr_os_imp_time_get
0001:00018a3c  _apr_os_exp_time_get
0001:00018a80  _apr_os_imp_time_put
0001:00018aac  _apr_os_exp_time_put
0001:00018af0  _apr_time_clock_hires
0001:00018af8  _apr_time_now
0001:00018b2c  _apr_time_exp_tz
0001:00018bd8  _apr_time_exp_lt
0001:00018c04  _apr_time_exp_gmt
0001:00018c30* _apr_unix_setup_time
0001:00018ca0  _apr_apr_time_to_os2_time
0001:00018d88  _apr_os2_time_to_apr_time
0001:00018e40  _apr_sleep
Module: U:\extras\lib\apr-1.lib(shm.o)
0001:00018eb0  _apr_shm_remove
0001:00018ebc  _apr_shm_baseaddr_get
0001:00018ec8  _apr_shm_pool_get
0001:00018ed4  _apr_os_shm_get
0001:00018ee8  _apr_os_shm_put
0001:00018f3c  _apr_shm_size_get
0001:00018f6c  _apr_shm_detach
0001:00018f94  _apr_shm_destroy
0001:00018fc0  _apr_shm_attach
0001:00019054  _apr_shm_create
Module: U:\extras\lib\apr-1.lib(thread.o)
0001:00019120  _apr_threadattr_detach_set
0001:00019130  _apr_threadattr_detach_get
0001:00019148  _apr_threadattr_stacksize_set
0001:00019158  _apr_threadattr_guardsize_set
0001:00019184  _apr_thread_detach
0001:00019198  _apr_os_thread_get
0001:000191ac  _apr_os_thread_equal
0001:000191c0  _apr_thread_pool_get
0001:000191cc  _apr_thread_once
0001:0001920c  _apr_threadattr_create
0001:00019250  _apr_os_thread_put
0001:0001929c  _apr_thread_once_init
0001:00019344  _apr_thread_data_set
0001:00019358  _apr_thread_data_get
0001:0001936c  _apr_thread_yield
0001:00019380  _apr_thread_join
0001:000193ec  _apr_thread_exit
0001:00019408  _apr_os_thread_current
0001:0001942c  _apr_thread_create
Module: U:\extras\lib\apr-1.lib(threadpriv.o)
0001:000194f0  _apr_threadkey_private_get
0001:00019504  _apr_threadkey_private_set
0001:00019518  _apr_os_threadkey_get
0001:0001952c  _apr_os_threadkey_put
0001:00019584  _apr_threadkey_data_set
0001:00019598  _apr_threadkey_data_get
0001:000195ac  _apr_threadkey_private_delete
0001:000195dc  _apr_threadkey_private_create
Module: U:\extras\lib\apr-1.lib(charset.o)
0001:0001965c  _apr_os_default_encoding
0001:00019668  _apr_os_locale_encoding
Module: U:\extras\lib\aprutil-1.lib(apr_queue.o)
0001:000196a0  _apr_queue_size
0001:000196ac  _apr_queue_interrupt_all
0001:000196f4  _apr_queue_term
0001:00019738  _apr_queue_trypop
0001:000197e4  _apr_queue_trypush
0001:00019888  _apr_queue_pop
0001:00019970  _apr_queue_push
0001:00019a58  _apr_queue_create
Module: U:\extras\lib\apr-1.lib(sha2_glue.o)
0001:00019b90  _apr_crypto_sha256_new
Module: U:\extras\lib\apr-1.lib(apr_random.o)
0001:00019c8c  _apr_random_after_fork
0001:00019cfc  _apr_random_barrier
0001:00019d10  _apr_random_secure_ready
0001:00019d28  _apr_random_insecure_ready
0001:00019e18  _apr_random_insecure_bytes
0001:00019e4c  _apr_random_secure_bytes
0001:00019eb4  _apr_random_add_entropy
0001:0001a150  _apr_random_init
0001:0001a298  _apr_random_standard_new
Module: U:\extras\lib\aprutil-1.lib(apr_reslist.o)
0001:0001a300  _apr_reslist_timeout_set
0001:0001a314  _apr_reslist_invalidate
0001:0001a364  _apr_reslist_acquired_count
0001:0001a5a0  _apr_reslist_release
0001:0001a610  _apr_reslist_acquire
0001:0001a7d4  _apr_reslist_destroy
0001:0001a920  _apr_reslist_create
Module: U:\extras\lib\aprutil-1.lib(apr_rmm.o)
0001:0001acc0  _apr_rmm_detach
0001:0001acc8  _apr_rmm_addr_get
0001:0001acd8  _apr_rmm_offset_get
0001:0001ace8  _apr_rmm_overhead_get
0001:0001acfc  _apr_rmm_free
0001:0001ae94  _apr_rmm_malloc
0001:0001afb4  _apr_rmm_destroy
0001:0001b0f8  _apr_rmm_realloc
0001:0001b194  _apr_rmm_calloc
0001:0001b2f0  _apr_rmm_attach
0001:0001b360  _apr_rmm_init
Module: U:\extras\lib\aprutil-1.lib(sdbm.o)
0001:0001b4d0  _apr_sdbm_rdonly
0001:0001b5a8  _apr_sdbm_nextkey
0001:0001b66c  _apr_sdbm_firstkey
0001:0001bbe4  _apr_sdbm_store
0001:0001bd70  _apr_sdbm_delete
0001:0001be2c  _apr_sdbm_fetch
0001:0001bed4  _apr_sdbm_close
0001:0001bf44  _apr_sdbm_open
0001:0001c0d8  _apu__sdbm_nullitem
Module: U:\extras\lib\aprutil-1.lib(sdbm_lock.o)
0001:0001c160  _apr_sdbm_unlock
0001:0001c19c  _apr_sdbm_lock
Module: U:\extras\lib\aprutil-1.lib(apr_sha1.o)
0001:0001d3a0  _apr_sha1_init
0001:0001d418  _apr_sha1_update_binary
0001:0001d528  _apr_sha1_update
0001:0001d534  _apr_sha1_final
0001:0001d610  _apr_sha1_base64
Module: U:\extras\lib\apr-1.lib(signals.o)
0001:0001d6c0  _apr_signal_init
0001:0001d6e0  _apr_signal_description_get
0001:0001d6fc  _apr_signal_unblock
0001:0001d748  _apr_signal_block
0001:0001d794  _apr_signal
0001:0001d7e8  _apr_proc_kill
Module: U:\extras\lib\apr-1.lib(apr_strnatcmp.o)
0001:0001da6c  _apr_strnatcmp
0001:0001da90  _apr_strnatcasecmp
Module: U:\extras\lib\apr-1.lib(apr_strings.o)
0001:0001dadc  _apr_strfsize
0001:0001dc70  _apr_off_t_toa
0001:0001dd14  _apr_ltoa
0001:0001dd88  _apr_itoa
0001:0001ddfc  _apr_strtoi64
0001:0001de30  _apr_atoi64
0001:0001de54  _apr_strtoff
0001:0001deb4  _apr_pstrcatv
0001:0001df30  _apr_pmemdup
0001:0001df70  _apr_pstrmemdup
0001:0001dfb4  _apr_pstrdup
0001:0001dffc  _apr_pstrcat
0001:0001e0c0  _apr_pstrndup
Module: U:\extras\lib\apr-1.lib(apr_strtok.o)
0001:0001e120  _apr_strtok
Module: U:\extras\lib\aprutil-1.lib(apr_strmatch.o)
0001:0001e2d0  _apr_strmatch_precompile
Module: U:\extras\lib\apr-1.lib(apr_tables.o)
0001:0001e3b0  _apr_is_empty_array
0001:0001e3cc  _apr_array_clear
0001:0001e3dc  _apr_array_pop
0001:0001e408  _apr_table_elts
0001:0001e410  _apr_is_empty_table
0001:0001e42c  _apr_table_clear
0001:0001e4b4  _apr_table_addn
0001:0001e53c  _apr_array_copy_hdr
0001:0001e57c  _apr_table_vdo
0001:0001e70c  _apr_table_unset
0001:0001e8cc  _apr_table_setn
0001:0001eae0  _apr_table_get
0001:0001eb9c  _apr_table_compress
0001:0001f034  _apr_table_do
0001:0001f05c  _apr_table_add
0001:0001f110  _apr_table_set
0001:0001f378  _apr_table_mergen
0001:0001f4a8  _apr_table_merge
0001:0001f694  _apr_table_copy
0001:0001f724  _apr_table_make
0001:0001f774  _apr_table_clone
0001:0001f7d0  _apr_array_make
0001:0001f818  _apr_array_pstrcat
0001:0001f90c  _apr_array_copy
0001:0001f990  _apr_array_cat
0001:0001fa44  _apr_table_overlap
0001:0001fb08  _apr_table_overlay
0001:0001fba0  _apr_array_append
0001:0001fbd0  _apr_array_push
Module: U:\extras\lib\apr-1.lib(thread_cond.o)
0001:0001fc60  _apr_thread_cond_create
0001:0001fc6c  _apr_thread_cond_wait
0001:0001fc78  _apr_thread_cond_timedwait
0001:0001fc84  _apr_thread_cond_signal
0001:0001fc90  _apr_thread_cond_broadcast
0001:0001fc9c  _apr_thread_cond_destroy
0001:0001fca8  _apr_thread_cond_pool_get
Module: U:\extras\lib\apr-1.lib(thread_mutex.o)
0001:0001fcc0  _apr_thread_mutex_pool_get
0001:0001fccc  _apr_thread_mutex_unlock
0001:0001fcec  _apr_thread_mutex_destroy
0001:0001fd48  _apr_thread_mutex_trylock
0001:0001fd70  _apr_thread_mutex_lock
0001:0001fd98  _apr_thread_mutex_create
Module: U:\extras\lib\aprutil-1.lib(apr_thread_pool.o)
0001:0001fe20  _apr_thread_pool_tasks_count
0001:0001fe2c  _apr_thread_pool_scheduled_tasks_count
0001:0001fe38  _apr_thread_pool_threads_count
0001:0001fe44  _apr_thread_pool_busy_count
0001:0001fe54  _apr_thread_pool_idle_count
0001:0001fe60* _apr_thread_pool_tasks_run_count
0001:0001fe6c* _apr_thread_pool_tasks_high_count
0001:0001fe78* _apr_thread_pool_threads_high_count
0001:0001fe84* _apr_thread_pool_threads_idle_timeout_count
0001:0001fe90  _apr_thread_pool_idle_max_get
0001:0001fe9c* _apr_thread_pool_idle_wait_get
0001:0001feac* _apr_thread_pool_idle_wait_set
0001:0001fed0  _apr_thread_pool_thread_max_get
0001:0001fedc  _apr_thread_pool_threshold_get
0001:0001fee8  _apr_thread_pool_threshold_set
0001:0001ff10  _apr_thread_pool_task_owner_get
0001:00020198  _apr_thread_pool_thread_max_set
0001:00020224  _apr_thread_pool_idle_max_set
0001:00020278  _apr_thread_pool_tasks_cancel
0001:000207bc  _apr_thread_pool_top
0001:000207f4  _apr_thread_pool_push
0001:0002082c  _apr_thread_pool_schedule
0001:00020f8c  _apr_thread_pool_destroy
0001:00021014  _apr_thread_pool_create
Module: U:\extras\lib\apr-1.lib(proc.o)
0001:000212c0  _apr_procattr_cmdtype_set
0001:000212d0  _apr_procattr_detach_set
0001:000212e0  _apr_procattr_child_errfn_set
0001:000212e8  _apr_procattr_error_check_set
0001:000212f0  _apr_procattr_addrspace_set
0001:000212f8  _apr_proc_detach
0001:00021304  _apr_procattr_user_set
0001:00021310  _apr_procattr_group_set
0001:0002131c  _apr_procattr_limit_set
0001:00021328  _apr_proc_wait_all_procs
0001:00021468  _apr_proc_wait
0001:00021698  _apr_procattr_dir_set
0001:000216f0  _apr_proc_create
0001:00021ff4  _apr_proc_fork
0001:0002205c  _apr_procattr_child_err_set
0001:00022138  _apr_procattr_child_out_set
0001:00022214  _apr_procattr_child_in_set
0001:000222f0  _apr_procattr_io_set
0001:00022414  _apr_procattr_create
Module: U:\extras\lib\apr-1.lib(otherchild.o)
0001:00022500  _apr_proc_other_child_alert
0001:00022568  _apr_proc_other_child_refresh
0001:00022614  _apr_proc_other_child_refresh_all
0001:00022644  _apr_proc_other_child_unregister
0001:00022694  _apr_proc_other_child_register
Module: U:\extras\lib\apr-1.lib(thread_rwlock.o)
0001:00022720  _apr_thread_rwlock_pool_get
0001:0002272c  _apr_thread_rwlock_destroy
0001:00022794  _apr_thread_rwlock_unlock
0001:00022800  _apr_thread_rwlock_trywrlock
0001:00022854  _apr_thread_rwlock_wrlock
0001:000228c0  _apr_thread_rwlock_tryrdlock
0001:00022918  _apr_thread_rwlock_rdlock
0001:00022970  _apr_thread_rwlock_create
Module: U:\extras\lib\apr-1.lib(timestr.o)
0001:00022a20  _apr_strftime
0001:00022a88  _apr_ctime
0001:00022e60  _apr_day_snames
0001:00022e30  _apr_month_snames
0001:00022c4c  _apr_rfc822_date
Module: U:\extras\lib\aprutil-1.lib(apr_uri.o)
0001:00022e80  _apr_uri_parse_hostinfo
0001:00022f64  _apr_uri_port_of_scheme
0001:00022fb4  _apr_uri_parse
0001:00023400  _apr_uri_unparse
Module: U:\extras\lib\apr-1.lib(userinfo.o)
0001:00023800  _apr_uid_name_get
0001:00023874  _apr_uid_get
0001:000238cc  _apr_uid_homepath_get
0001:00023934  _apr_uid_current
Module: U:\extras\lib\apr-1.lib(groupinfo.o)
0001:00023960  _apr_gid_get
0001:000239b4  _apr_gid_name_get
Module: U:\extras\lib\aprutil-1.lib(getuuid.o)
0001:00023a30  _apr_uuid_get
Module: U:\extras\lib\aprutil-1.lib(uuid.o)
0001:00023c7c  _apr_uuid_parse
0001:00023dcc  _apr_uuid_format
Module: U:\extras\lib\apr-1.lib(version.o)
0001:00023e70  _apr_version
0001:00023e9c  _apr_version_string
Module: U:\extras\lib\aprutil-1.lib(xlate.o)
0001:00023eb0  _apr_xlate_sb_get
0001:00023ec8  _apr_xlate_conv_byte
0001:00023eec  _apr_xlate_close
0001:00023f44  _apr_xlate_conv_buffer
0001:0002411c  _apr_xlate_open
Module: U:\extras\lib\aprutil-1.lib(apr_xml.o)
0001:000242f0  _apr_xml_insert_uri
0001:00024384  _apr_xml_empty_elem
0001:000243cc  _apr_xml_quote_string
0001:000244e8  _apr_xml_quote_elem
0001:00024594  _apr_text_append
0001:00024e1c  _apr_xml_to_text
0001:00024f78  _apr_xml_parser_geterror
0001:000250a0  _apr_xml_parser_done
0001:00025100  _apr_xml_parser_feed
0001:00025150  _apr_xml_parser_create
0001:00025270  _apr_xml_parse_file
Module: U:\extras\lib\aprutil-1.lib(apu_version.o)
0001:00025750  _apu_version
0001:0002577c  _apu_version_string
Module: U:\dev\httpd-2.2.17\server\.libs\main.lib(listen.o)
0001:00025790  _ap_listen_pre_config
0001:000257f8  _ap_set_receive_buffer_size
0001:0002588c  _ap_set_send_buffer_size
0001:000258fc  _ap_set_listenbacklog
0001:00025a3c  _ap_set_listener
0001:00025d88  _ap_close_listeners
0001:00026084  _ap_setup_listeners
0002:00002d50  _ap_listeners
Module: U:\dev\httpd-2.2.17\server\mpm\mpmt_os2\.libs\mpmt_os2.lib(mpmt_os2.o)
0002:00003dc0  _ap_server_conf
0001:000265d0  _ap_mpm_query
0001:00026668  _ap_graceful_stop_signalled
0001:00026cb8  _ap_mpm_run
0002:00001264* _ap_max_daemons_limit
0002:00001260  _ap_thread_stack_size
0002:00001270  _mpm_mpmt_os2_module
0002:00002da4  _ap_max_spare_threads
0002:00002da0  _ap_min_spare_threads
0002:00002da8  _ap_my_generation
0002:00002dac  _ap_mpm_accept_mutex
Module: U:\dev\httpd-2.2.17\os\os2\.libs\os.lib(util_os2.o)
0001:000279b0  _ap_os_create_privileged_process
Module: U:\dev\httpd-2.2.17\server\.libs\main.lib(provider.o)
0001:00027a0c  _ap_lookup_provider
0001:00027a78  _ap_list_provider_names
0001:00027b54  _ap_register_provider
Module: U:\dev\httpd-2.2.17\server\.libs\main.lib(util_pcre.o)
0001:00027d40  _ap_regfree
0001:00027d58  _ap_regexec
0001:00027f20  _ap_regcomp
0001:00027fc0  _ap_regerror
Module: U:\dev\httpd-2.2.17\server\.libs\main.lib(util_debug.o)
0001:00028120  _ap_get_module_config
0001:00028134  _ap_set_module_config
0001:00028148  _ap_strstr_c
0001:00028154  _ap_strstr
0001:00028160  _ap_strrchr_c
0001:0002816c  _ap_strrchr
0001:00028178  _ap_strchr_c
0001:00028184  _ap_strchr
Module: U:\dev\httpd-2.2.17\server\.libs\main.lib(config.o)
0001:00028190  _ap_hook_get_header_parser
0001:0002819c  _ap_run_header_parser
0001:000281f0  _ap_hook_get_pre_config
0001:000281fc  _ap_run_pre_config
0001:00028260  _ap_hook_get_test_config
0001:0002826c  _ap_run_test_config
0001:000282b4  _ap_hook_get_post_config
0001:000282c0  _ap_run_post_config
0001:00028328  _ap_hook_get_open_logs
0001:00028334  _ap_run_open_logs
0001:0002839c  _ap_hook_get_child_init
0001:000283a8  _ap_run_child_init
0001:000283f0  _ap_hook_get_handler
0001:000283fc  _ap_run_handler
0001:0002844c  _ap_hook_get_quick_handler
0001:00028458  _ap_run_quick_handler
0001:000284b0  _ap_hook_get_optional_fn_retrieve
0001:000284bc  _ap_run_optional_fn_retrieve
0001:00028500  _ap_find_module_name
0001:0002850c  _ap_set_config_vectors
0001:00028594  _ap_set_string_slot
0001:000285ac  _ap_set_flag_slot
0001:000285c8  _ap_set_deprecated
0001:000285ec  _ap_single_module_configure
0001:00028648  _ap_run_rewrite_args
0001:00028684  _ap_show_mpm
0001:000286ac  _ap_show_modules
0001:00028804  _ap_show_directives
0001:00028ab4  _ap_remove_module
0001:00028b40  _ap_remove_loaded_module
0001:00028ba0  _ap_merge_per_dir_configs
0001:00028c74  _ap_create_per_dir_config
0001:00028c80  _ap_create_conn_config
0001:00028c8c  _ap_create_request_config
0001:00028c98  _ap_set_string_slot_lower
0001:00028e5c  _ap_fixup_virtual_hosts
0001:00028fa0  _ap_init_virtual_host
0001:000290f0  _ap_find_linked_module
0001:00029bac  _ap_walk_config
0001:00029d34  _ap_process_config_tree
0001:00029e2c  _ap_find_command
0001:00029e74  _ap_find_command_in_modules
0001:00029ef8  _ap_soak_end_container
0001:0002a044  _ap_server_root_relative
0001:0002a0d0  _ap_set_file_slot
0001:0002a160  _ap_set_int_slot
0001:0002a5d4  _ap_build_config
0001:0002a8dc  _ap_parse_htaccess
0001:0002afec  _ap_process_resource_config
0001:0002b3a4  _ap_read_config
0001:0002b79c  _ap_build_cont_config
0001:0002b8d8  _ap_register_hooks
0001:0002ba40  _ap_add_module
0001:0002bb7c  _ap_setup_prelinked_modules
0001:0002bc6c  _ap_add_loaded_module
0001:0002bcb0  _ap_method_is_limited
0001:0002bd60  _ap_invoke_handler
0001:0002bf84  _ap_hook_optional_fn_retrieve
0001:0002c044  _ap_hook_quick_handler
0001:0002c0fc  _ap_hook_handler
0001:0002c1b8  _ap_hook_child_init
0001:0002c274  _ap_hook_open_logs
0001:0002c330  _ap_hook_post_config
0001:0002c3ec  _ap_hook_test_config
0001:0002c4a8  _ap_hook_pre_config
0001:0002c568  _ap_hook_header_parser
0002:00002e58  _ap_top_module
0002:00002e5c  _ap_loaded_modules
0002:00002e44  _ap_server_root
0002:00002e48  _ap_server_pre_read_config
0002:00002e4c  _ap_server_post_read_config
0002:00002e40  _ap_server_argv0
0002:00002e50  _ap_server_config_defines
0002:00002e54  _ap_conftree
Module: U:\dev\httpd-2.2.17\server\.libs\main.lib(util.o)
0001:0002c660  _ap_strcmp_match
0001:0002c720  _ap_strcasecmp_match
0001:0002c808  _ap_is_matchexp
0001:0002c838  _ap_strcasestr
0001:0002c928  _ap_stripprefix
0001:0002c964  _ap_getparents
0001:0002cb7c  _ap_no2slash
0001:0002cbc8  _ap_make_dirstr_prefix
0001:0002cc00  _ap_count_dirs
0001:0002cc2c  _ap_cfg_closefile
0001:0002cc4c  _ap_cfg_getc
0001:0002cc6c  _ap_size_list_item
0001:0002cd9c  _ap_find_list_item
0001:0002d298  _ap_escape_errorlog_item
0001:0002d3c0  _ap_is_url
0001:0002d418  _ap_str_tolower
0001:0002d43c  _ap_timeout_parameter_parse
0001:0002d51c  _ap_append_pid
0001:0002d550  _ap_escape_quotes
0001:0002d5f0  _ap_get_list_item
0001:0002d914  _ap_pcfg_open_custom
0001:0002d9e0  _ap_getword_conf
0001:0002db4c  _ap_getword_conf_nc
0001:0002db58  _ap_content_type_tolower
0001:0002db9c  _ap_ind
0001:0002dbd0  _ap_unescape_url_keep2f
0001:0002dd00  _ap_unescape_url
0001:0002de1c  _ap_escape_logitem
0001:0002df18  _ap_os_escape_path
0001:0002dff0  _ap_escape_path_segment
0001:0002e078  _ap_escape_shell_cmd
0001:0002e0ec  _ap_cfg_getline
0001:0002e344  _ap_pbase64encode
0001:0002e398  _ap_pbase64decode
0001:0002e4ac  _ap_get_local_host
0001:0002e6a0  _ap_rind
0001:0002e6d4  _ap_make_full_path
0001:0002e768  _ap_getword_white
0001:0002e80c  _ap_getword_white_nc
0001:0002e818  _ap_getword
0001:0002e8a4  _ap_getword_nc
0001:0002e8b8  _ap_make_dirstr_parent
0001:0002e918  _ap_is_rdirectory
0001:0002e954  _ap_is_directory
0001:0002e99c  _ap_escape_html2
0001:0002eb18  _ap_escape_html
0001:0002eb40  _ap_construct_server
0001:0002eb98  _ap_find_last_token
0001:0002ec18  _ap_find_token
0001:0002eca0  _ap_get_token
0001:0002ed84  _ap_getword_nulls
0001:0002edfc  _ap_getword_nulls_nc
0001:0002ee10  _ap_field_noparam
0001:0002eefc  _ap_pcfg_openfile
0001:0002f0f0  _ap_resolve_env
0001:0002f2d0  _ap_pregsub
0001:0002f484  _ap_pregfree
0001:0002f4b4  _ap_pregcomp
0001:0002f520  _ap_os_is_path_absolute
0001:0002f58c  _ap_ht_time
Module: U:\dev\httpd-2.2.17\server\.libs\main.lib(core.o)
0002:00003dd0  _ap_core_input_filter_handle
0002:00003de0  _ap_content_length_filter_handle
0002:00003df0  _ap_core_output_filter_handle
0002:00003e00  _ap_subreq_core_filter_handle
0002:00003e10  _logio_add_bytes_out
0001:0002f7d0  _ap_hook_get_get_mgmt_items
0001:0002f7dc  _ap_run_get_mgmt_items
0001:0002f898  _ap_allow_options
0001:0002f8c4  _ap_allow_overrides
0001:0002f8e0  _ap_auth_type
0001:0002f8fc  _ap_auth_name
0001:0002f924  _ap_default_type
0001:0002f94c  _ap_document_root
0001:0002f968  _ap_requires
0001:0002f984  _ap_satisfies
0001:0002f9a4  _ap_response_code_string
0001:0002f9f4  _ap_get_remote_logname
0001:0002fa1c  _ap_get_limit_req_body
0001:0002fa48  _ap_get_server_protocol
0001:0002fa60  _ap_set_server_protocol
0001:0002faac  _ap_get_server_revision
0001:0002fae4  _ap_get_server_description
0001:0002fb0c  _ap_get_server_banner
0001:0002fb24  _ap_get_server_version
0001:0002fb3c  _ap_get_limit_xml_body
0001:0002fb80  _ap_get_request_note
0001:000309e0  _ap_check_cmd_context
0001:0003197c  _ap_add_file_conf
0001:00031998  _ap_add_per_url_conf
0001:000319c0  _ap_add_per_dir_conf
0001:0003227c  _ap_custom_response
0001:000325b8  _ap_exists_config_define
0001:00035364  _ap_core_translate
0001:00033fb4  _ap_is_recursion_limit_exceeded
0001:00035134  _ap_register_request_note
0001:00035174  _ap_add_version_component
0001:00035558  _ap_add_output_filters_by_type
0001:00035618  _ap_limit_section
0001:000357b4  _ap_get_server_port
0001:0003584c  _ap_get_server_name
0001:00035944  _ap_psignature
0001:00035afc  _ap_construct_url
0001:00035c44  _ap_get_remote_host
0001:00035d60  _ap_core_reorder_directories
0001:00035e4c  _ap_hook_get_mgmt_items
0002:000012c0  _core_module
0002:000012b0  _ap_document_root_check
Module: U:\dev\httpd-2.2.17\server\.libs\main.lib(connection.o)
0001:00037650  _ap_hook_get_create_connection
0001:0003765c  _ap_run_create_connection
0001:000376d0  _ap_hook_get_process_connection
0001:000376dc  _ap_run_process_connection
0001:0003772c  _ap_hook_get_pre_connection
0001:00037738  _ap_run_pre_connection
0001:00037794  _ap_process_connection
0001:000377ec  _ap_flush_conn
0001:0003785c  _ap_lingering_close
0001:000378c0  _ap_hook_pre_connection
0001:00037984  _ap_hook_process_connection
0001:00037a48  _ap_hook_create_connection
Module: U:\dev\httpd-2.2.17\server\.libs\main.lib(eoc_bucket.o)
0001:00037b1c  _ap_bucket_eoc_make
0001:00037ba0  _ap_bucket_type_eoc
0001:00037b48  _ap_bucket_eoc_create
Module: U:\dev\httpd-2.2.17\server\.libs\main.lib(log.o)
0001:00037bd4  _ap_hook_get_error_log
0001:00037be0  _ap_run_error_log
0001:00037c5c  _ap_hook_error_log
0001:00037d0c  _ap_close_piped_log
0001:00037d84  _ap_logs_child_init
0001:00037db0  _ap_open_stderr_log
0001:00038374  _ap_log_cerror
0001:000383c8  _ap_log_perror
0001:00038420  _ap_log_error
0001:000387a8  _ap_open_piped_log_ex
0001:00038860  _ap_open_piped_log
0001:00038b20  _ap_log_assert
0001:00038bb8  _ap_read_pid
0001:00038d8c  _ap_log_pid
0001:00038f58  _ap_log_rerror
0001:00039020  _ap_error_log2stderr
0001:000390e0  _ap_replace_stderr_log
0001:00039788  _ap_open_logs
0002:00001300  _ap_default_loglevel
Module: U:\dev\httpd-2.2.17\modules\http\.libs\mod_http.lib(http_protocol.o)
0001:00039b60  _ap_hook_get_insert_error_filter
0001:00039b6c  _ap_run_insert_error_filter
0001:00039bc8  _ap_index_of_response
0001:00039c00  _ap_get_status_line
0001:00039c40  _ap_clear_method_list
0001:00039c60  _ap_copy_method_list
0001:00039ccc  _ap_make_method_list
0001:00039d1c  _ap_method_name_of
0001:00039f2c  _ap_send_http_options
0001:00039fe8  _ap_set_content_type
0001:0003b0a0  _ap_send_error_response
0001:0003bed4  _ap_method_number_of
0001:0003c410  _ap_method_list_remove
0001:0003c4cc  _ap_method_list_add
0001:0003c55c  _ap_method_in_list
0001:0003c64c  _ap_method_registry_init
0001:0003c950  _ap_method_register
0001:0003ca68  _ap_meets_conditions
0001:0003cdcc  _ap_set_keepalive
0001:0003d154  _ap_hook_insert_error_filter
Module: U:\dev\httpd-2.2.17\server\.libs\main.lib(protocol.o)
0001:0003d770  _ap_hook_get_post_read_request
0001:0003d77c  _ap_run_post_read_request
0001:0003d7d0  _ap_hook_get_log_transaction
0001:0003d7dc  _ap_run_log_transaction
0001:0003d830  _ap_hook_get_http_scheme
0001:0003d83c  _ap_run_http_scheme
0001:0003d88c  _ap_hook_get_default_port
0001:0003d898  _ap_run_default_port
0001:0003d8f8  _ap_hook_default_port
0001:0003d9b4  _ap_hook_http_scheme
0001:0003da74  _ap_hook_log_transaction
0001:0003db38  _ap_hook_post_read_request
0001:0003dc30  _ap_send_interim_response
0001:0003ddd8  _ap_rflush
0001:0003de3c  _ap_old_write_filter
0001:0003dff0  _ap_rvputs
0001:0003e0b8  _ap_rwrite
0001:0003e0f8  _ap_rputs
0001:0003e148  _ap_rputc
0001:0003e190  _ap_vrprintf
0001:0003e220  _ap_rprintf
0001:0003e254  _ap_send_fd
0001:0003e340  _ap_note_digest_auth_failure
0001:0003e3e0  _ap_note_auth_failure
0001:0003e490  _ap_note_basic_auth_failure
0001:0003e588  _ap_get_basic_auth_pw
0001:0003e780  _ap_finalize_request_protocol
0001:0003e7b4  _ap_finalize_sub_req_protocol
0001:0003e870  _ap_set_sub_req_protocol
0001:0003ea84  _ap_rationalize_mtime
0001:0003eac8  _ap_set_last_modified
0001:0003eb74  _ap_parse_uri
0001:0003ecd4  _ap_rgetline_core
0001:0003f1e0  _ap_get_mime_headers_core
0001:0003f644  _ap_read_request
0001:0003fef8  _ap_get_mime_headers
0001:0003ff34  _ap_getline
0001:0003ffb4  _ap_set_content_length
0001:00040030  _ap_content_length_filter
0001:0004027c  _ap_make_content_type
0001:000403b0  _ap_setup_make_content_type
0002:00002f90  _ap_old_write_func
Module: U:\dev\httpd-2.2.17\modules\http\.libs\mod_http.lib(http_etag.o)
0001:00040494  _ap_make_etag
0001:00040820  _ap_set_etag
Module: U:\dev\httpd-2.2.17\modules\http\.libs\mod_http.lib(http_filters.o)
0001:00040990  _ap_should_client_block
0001:000409d8  _ap_http_outerror_filter
0001:00040ab4  _ap_get_client_block
0001:00040cc8  _ap_setup_client_block
0001:00040f30  _ap_discard_request_body
0001:0004151c  _ap_basic_http_header
0001:00041800  _ap_http_header_filter
0001:000420dc  _ap_send_http_trace
0001:00042534  _ap_http_filter
Module: U:\dev\httpd-2.2.17\server\.libs\main.lib(error_bucket.o)
0001:000431f8  _ap_bucket_error_make
0001:000432d0  _ap_bucket_type_error
0001:00043270  _ap_bucket_error_create
Module: U:\dev\httpd-2.2.17\modules\http\.libs\mod_http.lib(byterange_filter.o)
0001:00043450  _ap_byterange_filter
Module: U:\dev\httpd-2.2.17\server\.libs\main.lib(request.o)
0001:00043ea0  _ap_hook_get_translate_name
0001:00043eac  _ap_run_translate_name
0001:00043efc  _ap_hook_get_map_to_storage
0001:00043f08  _ap_run_map_to_storage
0001:00043f58  _ap_hook_get_check_user_id
0001:00043f64  _ap_run_check_user_id
0001:00043fb4  _ap_hook_get_fixups
0001:00043fc0  _ap_run_fixups
0001:00044014  _ap_hook_get_type_checker
0001:00044020  _ap_run_type_checker
0001:00044070  _ap_hook_get_access_checker
0001:0004407c  _ap_run_access_checker
0001:000440d0  _ap_hook_get_auth_checker
0001:000440dc  _ap_run_auth_checker
0001:0004412c  _ap_hook_get_insert_filter
0001:00044138  _ap_run_insert_filter
0001:00044178  _ap_hook_get_create_request
0001:00044184  _ap_run_create_request
0001:00044244  _ap_update_mtime
0001:00044268  _ap_is_initial_req
0001:0004428c  _ap_destroy_sub_req
0001:000442a0  _ap_run_sub_req
0001:000445ac  _ap_some_auth_required
0001:00044638  _ap_sub_req_output_filter
0001:0004479c  _ap_file_walk
0001:00044a58  _ap_location_walk
0001:00045010  _ap_directory_walk
0001:00046200  _ap_process_request_internal
0001:00046510  _ap_sub_req_lookup_file
0001:00046734  _ap_sub_req_lookup_dirent
0001:00046b14  _ap_sub_req_method_uri
0001:00046c04  _ap_sub_req_lookup_uri
0001:00046c3c  _ap_hook_create_request
0001:00046cfc  _ap_hook_insert_filter
0001:00046dbc  _ap_hook_auth_checker
0001:00046e7c  _ap_hook_access_checker
0001:00046f3c  _ap_hook_type_checker
0001:00046ff4  _ap_hook_fixups
0001:000470b4  _ap_hook_check_user_id
0001:00047174  _ap_hook_map_to_storage
0001:00047234  _ap_hook_translate_name
Module: U:\dev\httpd-2.2.17\modules\http\.libs\mod_http.lib(http_request.o)
0001:000472f0  _ap_allow_standard_methods
0001:00047368  _ap_allow_methods
0001:000473b4  _ap_internal_fast_redirect
0001:000476cc  _ap_die
0001:00047e50  _ap_internal_redirect
0001:00047dd0  _ap_internal_redirect_handler
0001:00047ec8  _ap_process_request
Module: U:\dev\httpd-2.2.17\server\.libs\main.lib(vhost.o)
0001:00048060  _ap_vhost_iterate_given_conn
0001:000480f4  _ap_update_vhost_given_ip
0001:00048264  _ap_matches_request_vhost
0001:00048314  _ap_update_vhost_from_headers
0001:00048d34  _ap_set_name_virtual_host
0001:00048d64  _ap_init_vhost_config
0001:00048d9c  _ap_parse_vhost_addrs
0001:00049008  _ap_fini_vhost_config
Module: U:\dev\httpd-2.2.17\server\.libs\main.lib(mpm_common.o)
0001:00049710  _ap_hook_get_monitor
0001:0004971c  _ap_run_monitor
0001:000497a0  _ap_mpm_set_pidfile
0001:00049804  _ap_mpm_set_max_mem_free
0001:00049890  _ap_mpm_set_max_requests
0001:000498f0  _ap_gname2id
0001:00049984  _ap_uname2id
0001:00049a28* _ap_sock_disable_nagle
0001:00049ac0* _ap_mpm_safe_kill
0001:00049d54* _ap_relieve_child_processes
0001:00049df0* _ap_reclaim_child_processes
0001:00049fc0* _ap_unregister_extra_mpm_process
0001:0004a014* _ap_register_extra_mpm_process
0001:0004a044  _ap_hook_monitor
0002:00003430  _ap_pid_fname
0002:00003438  _ap_max_mem_free
0002:00003434  _ap_max_requests_per_child
Module: U:\dev\httpd-2.2.17\server\.libs\main.lib(scoreboard.o)
0001:0004a150  _ap_hook_get_pre_mpm
0001:0004a15c  _ap_run_pre_mpm
0001:0004a1b8  _ap_exists_scoreboard_image
0001:0004a1cc  _ap_get_scoreboard_worker
0001:0004a210  _ap_get_scoreboard_process
0001:0004a238  _ap_get_scoreboard_global
0001:0004a244  _ap_get_scoreboard_lb
0001:0004a26c  _ap_time_process_request
0001:0004a2cc  _ap_create_sb_handle
0001:0004a2f8* _find_child_by_pid
0001:0004a350  _ap_increment_counts
0001:0004a48c* _ap_cleanup_scoreboard
0001:0004a520* _ap_reopen_scoreboard
0001:0004a5d4  _ap_calc_scoreboard_size
0001:0004a6d4  _ap_init_scoreboard
0001:0004a8ac  _ap_create_scoreboard
0001:0004abcc  _ap_hook_pre_mpm
0001:0004ac84  _ap_update_child_status_from_indexes
0001:0004af04  _ap_update_child_status
0002:00003460  _ap_scoreboard_image
0002:00003464  _ap_scoreboard_fname
0002:00003468  _ap_extended_status
0002:0000346c  _ap_mod_status_reqtail
Module: U:\dev\httpd-2.2.17\server\.libs\main.lib(util_filter.o)
0001:0004afec  _ap_get_output_filter_handle
0001:0004b008  _ap_get_input_filter_handle
0001:0004b024  _ap_remove_input_filter
0001:0004b0a0  _ap_remove_output_filter
0001:0004b11c  _ap_get_brigade
0001:0004b174  _ap_pass_brigade
0001:0004b1c8  _ap_filter_protocol
0001:0004b1d8  _ap_fprintf
0001:0004b274  _ap_filter_flush
0001:0004b208  _ap_fputstrs
0001:0004b234  _ap_fflush
0001:0004b2a4  _ap_save_brigade
0001:0004b5d4  _ap_add_output_filter_handle
0001:0004b62c  _ap_add_input_filter_handle
0001:0004b7d8  _ap_add_output_filter
0001:0004b838  _ap_add_input_filter
0001:0004bbcc  _ap_register_output_filter_protocol
0001:0004bc04  _ap_register_output_filter
0001:0004bc34  _ap_register_input_filter
Module: U:\dev\httpd-2.2.17\server\.libs\main.lib(util_md5.o)
0001:0004bc70  _ap_md5contextTo64
0001:0004bd38  _ap_md5digest
0001:0004bdec  _ap_md5_binary
0001:0004be84  _ap_md5
Module: U:\dev\httpd-2.2.17\server\.libs\main.lib(util_script.o)
0001:0004c140  _ap_find_path_info
0001:0004c2ec  _ap_scan_script_header_err_core
0001:0004c820  _ap_scan_script_header_err_strs
0001:0004c87c  _ap_scan_script_header_err_brigade
0001:0004c8a8  _ap_scan_script_header_err
0001:0004c97c  _ap_add_cgi_vars
0001:0004cdc8  _ap_add_common_vars
0001:0004d364  _ap_create_environment
Module: U:\dev\httpd-2.2.17\server\.libs\main.lib(util_time.o)
0001:0004d648  _ap_explode_recent_gmt
0001:0004d67c  _ap_recent_rfc822_date
0001:0004d854  _ap_explode_recent_localtime
0001:0004d888  _ap_recent_ctime
Module: U:\dev\httpd-2.2.17\server\.libs\main.lib(util_xml.o)
0001:0004dad4  _ap_xml_parse_input
Module: U:\usr\lib\tcpipv4\libc_dll.lib(dllinit.obj)
0001:0004dd90  _DLL_InitTerm
Module: U:\usr\lib\libend.lib(src/libend/386/endlink386.asm)
0002:00003ea0  _end
0002:00002bd0  _edata
Module: U:\usr\lib\libend.lib(src/libend/386/end.asm)
0001:0007a740* _etext
0001:0007a740* __etext
0000:00000000* WEAK$ZERO
0002:00003ea0  __end
0002:00002bd0  __edata
Module: U:\dev\httpd-2.2.17\modules\http\.libs\mod_http.lib(http_core.o)
0002:00003e20  _ap_http_input_filter_handle
0002:00003e30  _ap_http_header_filter_handle
0002:00003e40  _ap_chunk_filter_handle
0002:00003e50  _ap_http_outerror_filter_handle
0002:00003e60  _ap_byterange_filter_handle
0002:00001320  _http_module
Module: U:\dev\httpd-2.2.17\modules\mappers\.libs\mod_so.lib(mod_so.o)
0002:00001360  _so_module
Module: U:\tmp\ldconv_gcc445_a_22764cbeb6951a4cb8.lib(__main.obj)
0001:0004efe0* ___do_global_ctors
0001:0004f017* ___do_global_dtors
0001:0004eff8  ___main
Module: U:\extras\lib\aprutil-1.lib(apu_dso.o)
0001:0004f070  _apu_dso_load
0001:0004f2e8  _apu_dso_init
0001:0004f3a8  _apu_dso_mutex_unlock
0001:0004f3c0  _apu_dso_mutex_lock
Module: U:\extras\lib\aprutil-1.lib(apr_dbm_sdbm.o)
0001:0004f710  _apr_dbm_type_sdbm
Module: U:\usr\lib\libos2.lib(code2.obj)
0001:0004f754  DosGetMessage
0001:0004f740* __msgseg32
Module: U:\extras\lib\apr-1.lib(maperrorcode.o)
0001:0004f7a4  _apr_canonical_error
Module: U:\extras\lib\apr-1.lib(filepath_util.o)
0001:0004f990  _apr_filepath_list_merge_impl
0001:0004fa7c  _apr_filepath_list_split_impl
Module: U:\extras\lib\apr-1.lib(os2calls.o)
0002:00003e70  _apr_os2_sendto
0002:00003e80  _apr_os2_recvfrom
0002:000013b0  _apr_os2_socket
0002:00003cc0  _apr_os2_select
0002:00003cc4  _apr_os2_sock_errno
0002:00003cc8  _apr_os2_accept
0002:00003ccc  _apr_os2_bind
0002:00003cd0  _apr_os2_connect
0002:00003cd4  _apr_os2_getpeername
0002:00003cd8  _apr_os2_getsockname
0002:00003cdc  _apr_os2_getsockopt
0002:00003ce0  _apr_os2_ioctl
0002:00003ce4  _apr_os2_listen
0002:00003ce8  _apr_os2_recv
0002:00003cec  _apr_os2_send
0002:00003cf0  _apr_os2_setsockopt
0002:00003cf4  _apr_os2_shutdown
0002:00003cf8  _apr_os2_soclose
0002:00003cfc  _apr_os2_writev
Module: U:\extras\lib\apr-1.lib(inet_pton.o)
0001:0004ffb0  _apr_inet_pton
Module: U:\extras\lib\apr-1.lib(inet_ntop.o)
0001:000500a0  _apr_inet_ntop
Module: U:\extras\lib\apr-1.lib(waitio.o)
0001:000501a0  _apr_wait_for_io_or_timeout
Module: U:\extras\lib\apr-1.lib(sha2.o)
0001:000502b0* _apr__SHA256_Transform
0001:00050504* _apr__SHA512_Transform
0001:00050c8c* _apr__SHA512_Last
0001:00050e6c* _apr__SHA384_Final
0001:00050f8c* _apr__SHA384_End
0001:00051040* _apr__SHA512_Final
0001:00051160* _apr__SHA512_End
0001:00051214  _apr__SHA256_Final
0001:000513d0* _apr__SHA256_End
0001:0005146c* _apr__SHA384_Init
0001:000514e8* _apr__SHA512_Update
0001:000516a4* _apr__SHA384_Update
0001:000516b0* _apr__SHA384_Data
0001:000516f8* _apr__SHA512_Init
0001:00051740* _apr__SHA512_Data
0001:000517bc  _apr__SHA256_Update
0001:000518dc  _apr__SHA256_Init
0001:00051914* _apr__SHA256_Data
Module: U:\extras\lib\aprutil-1.lib(sdbm_pair.o)
0001:00051d90  _apu__sdbm_fitpair
0001:00051dc4  _apu__sdbm_getnkey
0001:00051e10  _apu__sdbm_chkpage
0001:00051e80  _apu__sdbm_putpair
0001:00051eec  _apu__sdbm_splpage
0001:00052050  _apu__sdbm_delpair
0001:00052120  _apu__sdbm_duppair
0001:00052168  _apu__sdbm_getpair
Module: U:\extras\lib\aprutil-1.lib(sdbm_hash.o)
0001:000521c0  _apu__sdbm_hash
Module: U:\extras\lib\expat.lib(xmlparse.obj)
0001:00052323* _XML_UseParserAsHandlerArg
0001:0005232e* _XML_UseForeignDTD
0001:00052358* _XML_SetReturnNSTriplet
0001:0005237c  _XML_SetUserData
0001:00052397* _XML_GetBase
0001:000523a5* _XML_GetSpecifiedAttributeCount
0001:000523b3* _XML_GetIdAttributeIndex
0001:000523c1  _XML_SetElementHandler
0001:000523d5* _XML_SetStartElementHandler
0001:000523e3* _XML_SetEndElementHandler
0001:000523f1  _XML_SetCharacterDataHandler
0001:000523ff* _XML_SetProcessingInstructionHandler
0001:0005240d* _XML_SetCommentHandler
0001:0005241b* _XML_SetCdataSectionHandler
0001:0005242f* _XML_SetStartCdataSectionHandler
0001:0005243d* _XML_SetEndCdataSectionHandler
0001:0005244b  _XML_SetDefaultHandler
0001:00052460* _XML_SetDefaultHandlerExpand
0001:00052475* _XML_SetDoctypeDeclHandler
0001:00052489* _XML_SetStartDoctypeDeclHandler
0001:00052497* _XML_SetEndDoctypeDeclHandler
0001:000524a5* _XML_SetUnparsedEntityDeclHandler
0001:000524b3* _XML_SetNotationDeclHandler
0001:000524c1* _XML_SetNamespaceDeclHandler
0001:000524d5* _XML_SetStartNamespaceDeclHandler
0001:000524e3* _XML_SetEndNamespaceDeclHandler
0001:000524f1* _XML_SetNotStandaloneHandler
0001:000524ff* _XML_SetExternalEntityRefHandler
0001:0005250d* _XML_SetExternalEntityRefHandlerArg
0001:00052524* _XML_SetSkippedEntityHandler
0001:00052532* _XML_SetUnknownEncodingHandler
0001:00052549* _XML_SetElementDeclHandler
0001:0005255a* _XML_SetAttlistDeclHandler
0001:0005256b* _XML_SetEntityDeclHandler
0001:0005257c* _XML_SetXmlDeclHandler
0001:0005258d* _XML_SetParamEntityParsing
0001:000525b7* _XML_ParseBuffer
0001:000526e8* _XML_StopParser
0001:0005275f* _XML_ResumeParser
0001:00052848  _XML_GetErrorCode
0001:00052856* _XML_GetCurrentByteIndex
0001:00052875* _XML_GetCurrentByteCount
0001:00052897* _XML_GetInputContext
0001:000528c8* _XML_GetCurrentLineNumber
0001:00052921* _XML_GetCurrentColumnNumber
0001:00052977* _XML_FreeContentModel
0001:0005298c* _XML_MemMalloc
0001:000529a1* _XML_MemRealloc
0001:000529bc* _XML_MemFree
0001:000529d1  _XML_ErrorString
0001:000529f6* _XML_ExpatVersion
0001:00052a00* _XML_ExpatVersionInfo
0001:00052a1e* _XML_GetFeatureList
0001:00052b16* _XML_DefaultCurrent
0001:000532d9  _XML_ParserFree
0001:0005372a* _XML_GetParsingStatus
0001:00053770* _XML_GetBuffer
0001:000538f2  _XML_Parse
0001:00053c45* _XML_SetBase
0001:00053c8f* _XML_SetEncoding
0001:000556fa* _XML_ExternalEntityParserCreate
0001:00055d1d* _XML_ParserReset
0001:00056071* _XML_ParserCreate_MM
0001:000560be* _XML_ParserCreateNS
0001:000560e6  _XML_ParserCreate
Module: U:\dev\httpd-2.2.17\server\mpm\mpmt_os2\.libs\mpmt_os2.lib(mpmt_os2_child.o)
0002:00003e90+ _shutdown_event
0001:0005b9d4* thread_exception_handler
0001:0005bb90* _add_worker
0001:0005c198  _ap_mpm_child_main
Module: U:\dev\httpd-2.2.17\srclib\pcre\.libs\pcre.lib(pcre.o)
0001:0005c990* _pcre_version
0001:0005cb08  _pcre_info
0001:0005cb9c* _pcre_fullinfo
0001:0005cd30* _pcre_config
0001:00060388  _pcre_exec
0001:000638ac  _pcre_compile
0002:00002004  _pcre_free
0002:00002000* _pcre_malloc
0002:00002008* _pcre_stack_malloc
0002:0000200c* _pcre_stack_free
0002:00003d40* _pcre_callout
Module: U:\dev\httpd-2.2.17\server\.libs\main.lib(util_cfgtree.o)
0001:00065360  _ap_add_node
Module: U:\dev\httpd-2.2.17\server\.libs\main.lib(core_filters.o)
0001:000656e4  _ap_core_output_filter
0001:00066294  _ap_core_input_filter
Module: U:\usr\lib\tcpipv4\libc_dll.lib(syslog.obj)
0001:000667cc  _syslog
0001:00066834* _vsyslog
0001:00066c8c  _openlog
0001:00066cdc* _closelog
0001:00066d10* _setlogmask
Module: U:\tmp\ldconv_gcc445_a_22764cbeb6951a4cb8.lib(emx-ctordtor.obj)
0001:00066d40  ___ctordtorTerm
0001:00066d72  ___ctordtorInit
Module: U:\dev\httpd-2.2.17\modules\http\.libs\mod_http.lib(chunk_filter.o)
0001:00066dc0  _ap_http_chunk_filter
Module: U:\extras\lib\expat.lib(xmlrole.obj)
0001:00068a30  _XmlPrologStateInit
0001:00068a53  _XmlPrologStateInitExternalEntity
Module: U:\extras\lib\expat.lib(xmltok.obj)
0001:00077a4f  _XmlUtf8Encode
0001:00077aef* _XmlUtf16Encode
0001:00077b37  _XmlSizeOfUnknownEncoding
0001:00077d6c  _XmlInitUnknownEncoding
0001:00078292  _XmlGetUtf8InternalEncoding
0001:0007829c* _XmlGetUtf16InternalEncoding
0001:00078303  _XmlInitEncoding
0001:000783f5  _XmlParseXmlDecl
0001:00078445  _XmlGetUtf8InternalEncodingNS
0001:0007844f* _XmlGetUtf16InternalEncodingNS
0001:000784b6  _XmlInitEncodingNS
0001:000785a8  _XmlParseXmlDeclNS
0001:000785f8  _XmlInitUnknownEncodingNS
Module: U:\tmp\ldconv_gcc445_a_22764cbeb6951a4cb8.lib(emx-eh.obj)
0001:0007a535  ___ehInit
0001:0007a500* ___ehTerm
Module: U:\usr\lib\tcpipv4\libc_dll.lib(send.obj)
0001:0007a570* _send
Module: U:\usr\lib\tcpipv4\libc_dll.lib(connect.obj)
0001:0007a620* _connect
Module: U:\usr\lib\tcpipv4\libc_dll.lib(socket.obj)
0001:0007a6c0* _socket


                        +----------------------+
                        |   Imported Symbols   |
                        +----------------------+

Symbol                              Module
======                              ======

___libc_ForkRegisterModule          libc063
___init_dll                         libc063
___libc_Back_termDll                libc063
___libc_ForkDeregisterModule        libc063
__atfork_callback                   libc063
___stderrp                          libc063
__alloca                            libc063
___libc_GLocaleCtype                libc063
DosQueryProcAddr                    doscalls
DosFreeModule                       doscalls
DosLoadModule                       doscalls
DosQueryModuleHandle                doscalls
DosQueryPathInfo                    doscalls
DosSetPathInfo                      doscalls
DosFindFirst                        doscalls
DosQueryFileInfo                    doscalls
DosQueryHType                       doscalls
__errno                             libc063
DosDeleteDir                        doscalls
DosCreateDir                        doscalls
DosFindNext                         doscalls
DosFindClose                        doscalls
DosSetCurrentDir                    doscalls
DosSetDefaultDisk                   doscalls
DosQueryCurrentDisk                 doscalls
DosQueryCurrentDir                  doscalls
DosQueryFHState                     doscalls
DosSetFHState                       doscalls
DosMove                             doscalls
DosDelete                           doscalls
DosClose                            doscalls
DosOpen                             doscalls
DosSetFilePtr                       doscalls
DosSetRelMaxFH                      doscalls
DosWaitEventSem                     doscalls
DosWrite                            doscalls
DosSetFileLocks                     doscalls
DosRead                             doscalls
DosResetEventSem                    doscalls
DosDupHandle                        doscalls
DosSetFileSize                      doscalls
DosSetNPHState                      doscalls
DosCreateNPipe                      doscalls
DosConnectNPipe                     doscalls
DosCreateEventSem                   doscalls
DosSetNPipeSem                      doscalls
DosCloseEventSem                    doscalls
___stdoutp                          libc063
__assert                            libc063
___udivdi3                          libc063
getservbyname                       tcp32dll
gethostbyaddr                       tcp32dll
tcp_h_errno                         tcp32dll
gethostbyname                       tcp32dll
inet_addr                           tcp32dll
gethostname                         tcp32dll
___divdi3                           libc063
___threadid                         libc063
DosReleaseMutexSem                  doscalls
DosCloseMutexSem                    doscalls
DosRequestMutexSem                  doscalls
DosOpenMutexSem                     doscalls
DosCreateMutexSem                   doscalls
___moddi3                           libc063
DosSleep                            doscalls
DosGetSharedMem                     doscalls
DosQueryMem                         doscalls
DosFreeMem                          doscalls
DosGetNamedSharedMem                doscalls
DosAllocSharedMem                   doscalls
DosWaitThread                       doscalls
__endthread                         libc063
DosGetInfoBlocks                    doscalls
__beginthread                       libc063
DosFreeThreadLocalMemory            doscalls
DosAllocThreadLocalMemory           doscalls
_sys_siglist                        libc063
DosSendSignalException              doscalls
DosWaitChild                        doscalls
DosEnterCritSec                     doscalls
__getcwd2                           libc063
__chdir2                            libc063
DosExecPgm                          doscalls
DosExitCritSec                      doscalls
DosSearchPath                       doscalls
DosPostEventSem                     doscalls
_getpwuid_r                         libc063
_getpwnam_r                         libc063
_getgrnam_r                         libc063
_getgrgid_r                         libc063
DosQueryModuleName                  doscalls
_getpwnam                           libc063
__CRT_term                          libc063
__CRT_init                          libc063
__std_exit                          libc063
__std_fprintf                       libc063
__std_printf                        libc063
__std_puts                          libc063
__std_stricmp                       libc063
__std_strnicmp                      libc063
__std_free                          libc063
__std_malloc                        libc063
__std_memchr                        libc063
__std_strchr                        libc063
__std_atoi                          libc063
__std_strcat                        libc063
__std_sprintf                       libc063
__std_unsetenv                      libc063
__std_setenv                        libc063
__std_getenv                        libc063
DosTrueGetMessage                   msg
__std_strerror                      libc063
__std_strerror_r                    libc063
__std_fstat                         libc063
__std_access                        libc063
__std_strncmp                       libc063
__std_memcmp                        libc063
__std_close                         libc063
__std_unlink                        libc063
__std_write                         libc063
__std_lseek                         libc063
__std_writev                        libc063
__std_getpid                        libc063
__std_mkstemp                       libc063
__std_setmode                       libc063
__std_fcntl                         libc063
__std_strrchr                       libc063
__std_random                        libc063
__std_fwrite                        libc063
__std_fputc                         libc063
__std_fputs                         libc063
__std_qsort                         libc063
__std_strcmp                        libc063
__std_modf                          libc063
__std_getpass                       libc063
__std_strcpy                        libc063
__std_strncat                       libc063
__std_crypt                         libc063
__std_strtol                        libc063
__std_strspn                        libc063
__std_gettimeofday                  libc063
__std_gmtime_r                      libc063
__std_timezone                      libc063
__std_mktime                        libc063
__std_difftime                      libc063
__std_localtime                     libc063
__std_nl_langinfo                   libc063
__std_sigemptyset                   libc063
__std_sigaddset                     libc063
__std_sigprocmask                   libc063
__std_sigaction                     libc063
__std_kill                          libc063
__std_strtoll                       libc063
__std_waitpid                       libc063
__std_strpbrk                       libc063
__std_chdir                         libc063
__std_fork                          libc063
__std_strftime                      libc063
__std_getuid                        libc063
__std_getgid                        libc063
__std_srand                         libc063
__std_rand                          libc063
__std_iconv_close                   libc063
__std_iconv                         libc063
__std_iconv_open                    libc063
__std_signal                        libc063
__std_getppid                       libc063
__gettid                            libc063
DosUnwindException                  doscalls
DosSetExceptionHandler              doscalls
DosOpenQueue                        quecalls
DosReadQueue                        quecalls
DosQueryQueue                       quecalls
DosWriteQueue                       quecalls
DosSetSignalExceptionFocus          doscalls
DosCreateQueue                      quecalls
DosPurgeQueue                       quecalls
DosKillThread                       doscalls
__std_remove                        libc063
__std_strncpy                       libc063
__std_strstr                        libc063
__std_putchar                       libc063
__std_atol                          libc063
__std_time                          libc063
__std_ctime_r                       libc063
__getprogname                       libc063
__std_vsnprintf                     libc063
__std_open                          libc063
__std_memset                        libc063
__std_abort                         libc063
__std_freopen                       libc063
__std_sscanf                        libc063
__std_getgrnam                      libc063
__std_getpgid                       libc063
__std_getpgrp                       libc063
__std_times                         libc063
__std_calloc                        libc063
___ctordtorTerm1                    libc063
___ctordtorInit1                    libc063
__std_atexit                        libc063
__std_memmove                       libc063
__std_memcpy                        libc063
__std_realloc                       libc063
___deregister_frame                 libc063
___register_frame_table             libc063
___libc_FH                          libc063
__libsocket_set_errno               so32dll
__libsocket_send                    so32dll
__libsocket_sock_errno              so32dll
__libsocket_connect                 so32dll
__libsocket_socket                  so32dll
___libc_TcpipAllocFH43              libc063
__libsocket_soclose                 so32dll


                        +--------------------+
                        |   Libraries Used   |
                        +--------------------+

U:\dev\httpd-2.2.17\server\.libs\main.lib
U:\dev\httpd-2.2.17\modules\http\.libs\mod_http.lib
U:\dev\httpd-2.2.17\modules\mappers\.libs\mod_so.lib
U:\dev\httpd-2.2.17\server\mpm\mpmt_os2\.libs\mpmt_os2.lib
U:\dev\httpd-2.2.17\os\os2\.libs\os.lib
U:\dev\httpd-2.2.17\srclib\pcre\.libs\pcre.lib
U:\extras\lib\aprutil-1.lib
U:\extras\lib\expat.lib
U:\extras\lib\apr-1.lib
U:\usr\lib\libc_alias.lib
U:\usr\lib\tcpipv4\libc_dll.lib
U:\usr\lib\libos2.lib
U:\tmp\ldconv_gcc445_a_22764cbeb6951a4cb8.lib
U:\usr\lib\libend.lib


                        +-----------------------+
                        |   Linker Statistics   |
                        +-----------------------+

Stack size:  0000 (0.)
Memory size:  0007e5e0 (517600.)
Link time: 00:00.09
